:020000040800F2
:1080000000A000206940010825FC000827FC0008AA
:1080100029FC00082BFC00082DFC000800000000D3
:108020000000000000000000000000002FFC00081D
:1080300031FC00080000000033FC0008F581000856
:10804000AD400108AD400108AD400108AD40010858
:10805000AD400108AD400108AD400108AD40010848
:10806000AD400108AD400108AD400108AD40010838
:10807000AD400108AD400108AD400108AD40010828
:10808000AD400108AD400108AD400108AD40010818
:10809000AD400108AD400108AD40010891870008DE
:1080A000AD400108AD400108AD400108AD400108F8
:1080B000AD400108E7EF0008AD400108AD40010800
:1080C000AD400108AD400108AD4001082DEC0008AD
:1080D000AD400108998A0008AD400108AD40010893
:1080E000AD400108AD400108AD400108AD400108B8
:1080F000AD400108AD400108AD400108AD400108A8
:10810000000000000000000000000000AD40010879
:10811000AD400108AD400108AD400108AD40010887
:10812000AD400108AD400108AD400108AD40010877
:10813000AD400108AD400108000000000000000053
:10814000AD400108AD400108AD400108000000004D
:10815000000000000000000000000000000000001F
:108160000000000000000000AD400108AD40010823
:10817000AD40010800000000000000000000000009
:0881800000000000AD40010801
:1081880010B5054C237833B9044B13B10448AFF349
:1081980000800123237010BDA4000020000000000F
:1081A800888100080C4B43B10C480D4910B5AFF35A
:1081B80000800C48036823B910BD0A48036833B926
:1081C8007047094B002BF7D0BDE810401847064B05
:1081D800002BF5D0184700BF000000008881000878
:1081E800A8000020A400002000000000684620F03D
:1081F80007018D4619B51A4B1A781C46002A2CD04F
:108208005B68184A01336360136801331360164BC7
:108218001A6812B11A68013A1A60144B1A685AB1EE
:108228001A68013A1A601B6833B9114B1B681BB1F5
:10823800104B187800F0C6F9002323700E4B1A680B
:108248003AB11A68013A1A601B6813B90B4B01223C
:108258001A70BDE819408546704701221A70EDE78B
:10826800C000002004300020402E0020882E00206E
:10827800642E0020922F0020442E0020482E00203B
:108288000A4B10B541F29312094C5A60F02284F857
:10829800232000229A6007221A606FF0040009F078
:1082A8002FF8302384F8233010BD00BF10E000E021
:1082B80000ED00E0014B5868704700BFC000002087
:1082C80038B5002205460C460220CF2100F0A8FD53
:1082D80029460022022000F0A3FD214601220220A7
:1082E800BDE8384000F09CBD08B5012009F04EFFFC
:1082F800000A05280AD1012009F048FFC0B25A280F
:1083080004D10220BDE8084009F040BF002008BDA4
:108318000020704708B5012009F038FF000A052839
:1083280001D0002008BD012009F030FFC0B25A2852
:10833800F7D1032009F02AFF000A431E584258418A
:1083480008BD002070472DE9F041012186B04FF4A7
:108358000030002409F038FA032640F6430302A946
:108368004FF0904001274FF0904502938DF80D6033
:108378008DF80C408DF80E408DF80F4008F040FD48
:1083880049F2BC0302A94FF0904002938DF80C709B
:108398008DF80D608DF80E408DF80F4008F030FD17
:1083A80048F21803AB61A023AB614FF4807302A9B4
:1083B800029328460223DFF8C0818DF80C308DF82F
:1083C8000D608DF80E408DF80F4008F019FD06205D
:1083D80009F028F839464FF4802009F0F5F94046AD
:1083E80041F2032302A902938DF80D608DF80C4029
:1083F8008DF80E408DF80F4008F002FD404640F61B
:10840800045302A902938DF80C708DF80D608DF855
:108418000E408DF80F4008F0F3FC40F60403C8F84E
:1084280018304FF0A063C8F81830394608F580684E
:108438004FF4002009F0C8F94FF46043404602A900
:1084480002938DF80C708DF80D608DF80E408DF844
:108458000F4008F0D5FC4FF06043C8F81830444B83
:108468008DF80C704FF4005802A928461C708DF83E
:108478000D60CDF808808DF80E408DF80F4008F09B
:10848800BFFC4FF4804302A9284602938DF80D6083
:108498008DF80F708DF80C408DF80E404FF0005796
:1084A80008F0AEFC2E460A2122464346AF614FF43F
:1084B8007A7000BF0138FCD1288AB361400458BFE4
:1084C80001324FF47A7000BF0138FCD1288A400489
:1084D80048BF01340139E9D10A2A264B46D10A2C72
:1084E80044D101221A704FF4C0430024029302269B
:1084F800032302A94FF090408DF80D308DF80C60E1
:108508008DF80E408DF80F4008F07AFC22460D21B8
:108518004FF0904008F0ECFC22460E214FF09040BE
:1085280008F0E6FC144B4FF480629A6108210120A0
:108538000AF004F90823049301250C2304A88DF8F4
:1085480015308DF814408DF8165008F089F8172367
:1085580001A88DF804308DF805608DF806408DF877
:10856800075008F089FE06B0BDE8F0810022B9E79F
:10857800C8000020802E00200004004837B50F4BAB
:108588001B78C3B10E484FF090424FF400250021EC
:10859800082495610191019B834208D99461019156
:1085A800019B8342F5D8019B01330193F8E7019BB6
:1085B80001330193EFE703B030BD00BF802E0020E8
:1085C8003F0D030001280E4B0ED008D302280FD010
:1085D8001A784FF090437AB104229A6170471A785A
:1085E80022F001021A70F3E71A7822F00202F9E782
:1085F8001A7822F00402F5E74FF48022EDE700BF75
:10860800C800002001280E4B0ED008D302280FD036
:108618001A784FF090437AB104229A6170471A7819
:1086280042F001021A70F3E71A7842F00202F9E701
:108638001A7842F00402F5E74FF48022EDE700BF14
:10864800C800002010B50021044644FA01F3DB07F6
:10865800C8B205D5FFF7D6FF01310829F5D110BDFD
:10866800FFF7B0FFF8E718B1012807D000207047DE
:108678004FF09043188A00F0010070474FF0904384
:10868800188AC0F3C0207047012809D003D30228F4
:108698000BD000207047074B187800F00100704796
:1086A800044B1878C0F340007047024B1878C0F3A9
:1086B80080007047C80000204FF09043188A1B8A3A
:1086C80000F001001B0548BF40F002007047064B50
:1086D8001B7803F001009A0748BF40F002005B07CF
:1086E80048BF40F004007047C800002070470120D0
:1086F8007047034B10B1034ADA607047024AFBE740
:1087080000ED00E00400FA050100FA0500224FF030
:10871800FF31930003F1604303F561430132082AF6
:10872800C3F88010C3F88011F3D100230448194618
:10873800C2180133F02B82F80013F9D1704700BF3B
:1087480000E100E0C0B201F0A3B9C0B201F092B9F3
:10875800C0B201F0ABB9024B4FF400629A617047A6
:1087680000040048024B4FF000629A61704700BF56
:1087780000040048034B988A80F40060C0F3C020CE
:10878800704700BF00040048684620F007018D4686
:1087980019B5082008F00CF8012801460ED1094C3B
:1087A800236843B1084B1878FFF72CFF074B226862
:1087B8001A60074B1970082008F00DF8BDE8194039
:1087C80085467047642E0020922F0020882E0020B6
:1087D800912F00202DE9F04385B081468846414815
:1087E8009DF830404FF480511E46174609F08DFE23
:1087F8004FF4E0613B4809F080FE0022B0210220DE
:1088080000F00EFB01228321022000F009FB364B09
:10881800002201ADA3F10C01B9F1000F5FD0505C4B
:10882800A85401320C2AF7D1B9F1000F28D19DF8CC
:1088380008109DF8092008F07F0321F07F011943F3
:108848008DF808109DF80D1006F07F0321F07F01C8
:108858000B438DF80D309DF80A3003F00F0343EAFF
:10886800041322F07F0207F07F073A438DF80A309D
:10887800E3064CBF62F07F0202F07F028DF8092008
:1088880000270224E95DF8B20B46082684EA0302B1
:10889800640012F0800FE4B206F1FF3618BF84F0CE
:1088A8001D045B0016F0FF06DBB2EFD10137FFF7BE
:1088B80007FD0C2FE6D121463846FFF701FD0121BF
:1088C8007420FFF7FDFC3146064809F01EFE0548F6
:1088D8004FF4706105B0BDE8F04309F00EBED05CFE
:1088E8009EE700BF003C0040AA41010830B504469D
:1088F8008BB05D480AF01EFD01214FF4804008F05E
:108908006FFF01214FF4003008F05EFF4FF4B053C1
:108918000293022303228DF80C3002A900234FF0A2
:1089280090408DF80E308DF80F308DF80D2008F03E
:1089380067FA072209214FF0904008F0D9FA072278
:108948000A214FF0904008F0D3FA07220C214FF08B
:10895800904008F0CDFA44480AF0ECFC04A80AF06C
:1089680093FD0B2C7DD8DFE804F07C066164676A10
:108978006D707376787A4FF4615304A93A4804937A
:108988000AF026FD002138480AF0AAFE08213648D8
:108998000AF0AEFE082134480AF0B3FE012132483D
:1089A8000AF095FE2523002401258DF8043001A83E
:1089B80006238DF805308DF806408DF8075008F02D
:1089C8005BFC40F2FF3128480AF0E3FE22464FF4F0
:1089D800847125480AF0AEFE2A46244922480AF046
:1089E800A9FE2246224920480AF0A4FE2A46214927
:1089F8001D480AF09FFE22461F491B480AF09AFEAE
:108A080022461E4918480AF095FE22461C49164877
:108A18000AF090FE22464FF4407113480AF08AFE8D
:108A2800294611480AF04FFD0BB030BD4FF496436C
:108A3800A3E74FF4E143A0E74FF416439DE74FF453
:108A480061439AE74FF4963397E74FF4E13394E79D
:108A58004FF4613391E70B4B8FE70B4B8DE70B4BD3
:108A68008BE74FF4165388E70038014007010700E9
:108A780006010600050105000401040006020800BD
:108A88000A03090090D0030020A1070040420F000C
:108A9800684620F007018D4619B5244924480AF094
:108AA8007AFEC8B1234A22491368898C5068013379
:108AB800B3F5905F08BF0023834289B204D01068E1
:108AC8001044C9B2017213601B4B0A221A601B4B77
:108AD800D3F810211A4B1A60154C1A4920460AF08F
:108AE8005AFEC8B1164B1A68B2B9144BD3F8140120
:108AF800D3F81811884213D0D3F81811481C194418
:108B0800C3F8180191F81C112185D3F81811B1F593
:108B1800905F01D1C3F81821BDE819408546704718
:108B2800084920460AF006FEF6E700BF05010500E1
:108B380000380140CC000020442E0020C411002041
:108B4800402E0020070107000C4AD2F81431D2F851
:108B580018110133B3F5905F08BF00238B420BD087
:108B6800D2F81411114481F81C01C2F814310449D7
:108B7800044801220AF0DEBD704700BFC41100207E
:108B880007010700003801400A4B59681A689142EA
:108B98000DD05A68511C1A445960127A02705A68EA
:108BA800B2F5905F01D100225A6001207047002081
:108BB800704700BFCC000020014BC3F8100170477C
:108BC800C4110020044B1A7802F0FF0012B10022F1
:108BD8001A700120704700BF482E002072B6034B60
:108BE80000225A601A6062B6704700BFCC000020AD
:108BF80010B5441E14F8010F00B910BDFFF7A4FF0B
:108C0800F8E700BFF0B5012189B04FF4004008F043
:108C1800F3FD002438230227032601214FF4802086
:108C280001938DF808708DF80A408DF809608DF869
:108C38000B4008F0C9FD01A9754808F0E1F80622C3
:108C48003146734808F054F906220421704808F0A8
:108C58004FF9062205216E4808F04AF96D4809F0D7
:108C68003FFB4FF48273ADF80E304FF4E063ADF87C
:108C780010304FF400730125ADF8163003A908230E
:108C88006448ADF81830ADF80C40ADF81270ADF886
:108C98001450ADF81A40ADF81C4009F061FB4FF4D0
:108CA80080515C4809F031FC29465A4809F001FC1A
:108CB800FFF72EFB002850D029464FF4804008F0DB
:108CC8009BFD4FF4704329464FF4802001938DF8A3
:108CD80008708DF80A408DF809608DF80B4008F08F
:108CE80073FD01A94A4808F08BF805220C21484871
:108CF80008F0FEF805220D21454808F0F9F805228C
:108D08000E21434808F0F4F805220F21404808F0E6
:108D1800EFF8414809F0E4FA4FF47063ADF8103009
:108D280003A910233C48ADF81830ADF80C40ADF855
:108D38000E40ADF81240ADF81450ADF81640ADF83D
:108D48001A40ADF81C4009F00BFB2146324809F0E7
:108D5800DCFB2946304809F0ACFB01214FF4805078
:108D680008F03EFDE023002401930225032301219E
:108D78004FF400308DF809308DF808508DF80A400E
:108D88008DF80B4008F020FD01A94FF0904008F045
:108D980037F8052211464FF0904008F0A9F805224F
:108DA80006214FF0904008F0A3F8052207214FF064
:108DB800904008F09DF8194809F092FA4FF4827330
:108DC800ADF80E304FF4E063ADF810304FF4007397
:108DD800ADF81250ADF816300125182303A90F4835
:108DE800ADF81830ADF80C40ADF81450ADF81A4095
:108DF800ADF81C4009F0B4FA4FF48051074809F067
:108E080084FB2946054809F054FB09B0F0BD00BFB2
:108E180000040048003C0040003800400030014099
:108E28000128F8B505460E4614462AD003D3022871
:108E38002CD00020F8BD2A4B4FF48022294F9A618C
:108E48000221384609F01BFC0028F9D0F1B2254868
:108E5800244E09F0BCFB0121304609F010FC002823
:108E6800F9D0002C36D0012D2FD029D3022DE0D1F6
:108E78004FF0904310229A611B4809F0ACFB80B276
:108E8800F8BD4FF000424FF09043D7E74FF09043C2
:108E98004FF48012144D9A610221284609F0EFFB25
:108EA8000028F9D0F1B210480F4D09F090FB0121CC
:108EB800284609F0E4FB0028F9D0002CDCD0D7E7DD
:108EC800074B04229A610748D7E74FF400424FF056
:108ED8009043F7E7012DF6D9022DAAD1CCE700BFC0
:108EE8000004004800300140003C004010B5FFF786
:108EF800E1F90446FFF7DEF9001B0028B8BF40423D
:108F08000628F7DD10BD07B5030A8DF804308DF883
:108F180005008DF80610A023032201A9034806F0D6
:108F280046FEFFF7E3FF03B05DF804FB0054004082
:108F38002DE9F0411546154F00228AB00E46144619
:108F4800AC4202D10AB0BDE8F0810AAB1344315DEE
:108F580003F8221C531C00EB030818F01F0F02D063
:108F6800691E8C420ED1030A8DF804308DF8050075
:108F7800A023033201A9384606F019FEFFF7B6FF11
:108F88004046002301341A46DAE700BF0054004087
:108F980013B50B4C8DF80500030A8DF8043001A9B0
:108FA800A0230222204606F002FEA023022201A9E5
:108FB800204606F0C5FD9DF8040002B010BD00BFB4
:108FC8000054004073B50B4C8DF80500030A0D469C
:108FD80016468DF8043001A9A0230222204606F087
:108FE800E6FDA02332462946204606F0A9FD02B038
:108FF80070BD00BF00540040C0EBC000072200F560
:109008000060FFF795BFC0EBC000072200F50060C5
:10901800FFF7D8BF70B500238AB001AD1A465A557C
:109028000133222BFBD10B4E4FF40064230A8DF839
:1090380004308DF80540A0232222294630462034EA
:1090480006F0B5FDFFF752FFB4F5005FEED10AB0A8
:1090580070BD00BF0054004013B50C46C0EBC00003
:109068000722694600F50060FFF7ACFF9DF8002075
:1090780023789A4212D19DF8012063789A420DD143
:109088009DF80220A3789A4208D1DDF80300D4F8AD
:109098000330C31A5842584102B010BD0020FBE704
:1090A800704737B540F2FF70FFF772FF2A2802D1E8
:1090B800254B1B788BB3002140F2FF70FFF723FF8D
:1090C800FFF7A8FF402221490020FFF731FF402287
:1090D8001F49104602ADFFF72BFF002345F8043D5A
:1090E8004FF4C3642046042229460434FFF720FFC6
:1090F800B4F5FF6FF6D1002301934FF4A76420461F
:10910800042229460434FFF713FFB4F5C36FF6D1E0
:109118002A2140F2FF70FFF7F6FE40220B4900209B
:10912800FFF750FF402210460A49FFF74BFFFFF7B1
:10913800EFF84C2228B9084908480BF021F803B089
:1091480030BD0749F8E700BF802E0020040000204A
:1091580050420108902E0020B8410108D02E00206E
:109168000442010838B56FF0007204460D460C2120
:1091780000F0F1FC0E21204600F00DFD2A466C217E
:10918800204600F0E8FC0E21204600F004FD830193
:10919800F9D56E21204600F0FEFC014B186038BD61
:1091A800E024002010B5404C0B2303FB004203FBD6
:1091B80000431179032984BF032111719A79032A85
:1091C80084BF03229A710B2303FB004203FB004375
:1091D800117A0F2984BF0F2111725A7A072A84BF86
:1091E80007225A720B2303FB004203FB0043917AC8
:1091F8000F2984BF0F2191725A7B0F2A84BF0F2237
:109208005A730B2303FB004203FB0043917B0F2996
:1092180084BF0F2191731A79D20342F4002121618E
:10922800597911B142F4042222610B2303FB004354
:10923800DB791BB1236943F4005323610B2202FB42
:109248000042C9B9137A9179527ADB0143EAC12302
:1092580021690B4343EA021323610B2303FB0043F9
:10926800DA7A1AB922699B7A134323612169FFF7D5
:1092780079FF2369636110BD137B1BB1236943F434
:10928800805323610B2303FB0043997B5A7B23699B
:1092980043EAC2130A0102F0700213430A0748BFE7
:1092A80043F40063D8E700BFE024002038B51D4C24
:1092B8004FF46023C2002361A318DB7F13B14FF47E
:1092C80070232361A1184B7E0D7E897E1B0343EA20
:1092D80085332569012943EA0503236104EB02016B
:1092E80004BF43F4806323612369CD7E097F43EA89
:1092F80005230129236104BF43F080032361A318D8
:1093080022445B7F012B02BF236943F040032361A2
:109318002169937F41EA03112161FFF723FF236944
:10932800236238BDE024002010B54300254C1A18EC
:10933800224492F925103F29C4BF3F2182F8251005
:109348001A18224492F925103F31BCBFC12182F876
:1093580025101A18224492F826101F2984BF1F21AD
:1093680082F826104FF4402222611A18224492F8FB
:109378002420012A04BF4FF45022226104EBC002CA
:10938800D17F1A18224492F8252089B9120221693E
:1093980002F4FE420A4303442344226193F8261050
:1093A800236919432161FFF7DDFE2369A36210BD1C
:1093B80001F0030102F07C020A43216941EA02221A
:1093C800E9E700BFE024002010B58300244C1A18F8
:1093D800224492F82C10012984BF012182F82C1014
:1093E8001A18224492F82D10032984BF032182F809
:1093F8002D101A18224492F82E100F2984BF0F211D
:1094080082F82E101A18224492F82F10032984BFCC
:10941800032182F82F101A182244034492F83010BE
:109428000F29234484BF0F2182F8301093F830109D
:1094380093F82C2041F4202141EAC23193F82D20E1
:1094480041EA423193F82E2093F82F3041EA022165
:1094580041EA43112161FFF785FE2369636310BD6B
:10946800E024002010B5134C00232361C300E21848
:1094780092F83D2012B14FF400722261E21892F87E
:109488003E201AB1226942F480722261E218234414
:1094980092F83F100F2984BF0F2182F83F1093F8EC
:1094A8003F10236919432161FFF75CFE2369236498
:1094B80010BD00BFE0240020204B052210B501217B
:1094C80083F825201F22002483F8241083F82620FF
:1094D80019770322597702219C76DC76DC7783F8AA
:1094E8002C4083F82D4083F82E4083F82F4083F8D2
:1094F800304083F83D4083F83E4083F83F405C713C
:10950800DC719C71DC721C735C731A765A769977DD
:10951800197119725A729A729A732046FFF7A2FF4C
:109528002046FFF751FF2046FFF7FEFE2046FFF7D3
:10953800BDFE2046BDE8104034E600BFE024002010
:10954800054B042903EBC00318BF002283F83F1022
:1095580018BF83F83D2085E7E0240020044B03EB87
:10956800C00383F83D1011B1042283F83F2079E746
:10957800E0240020024B03EBC00383F83E1071E7A0
:10958800E0240020024B03EBC00090F83F00704736
:10959800E0240020024B03EBC00090F83D00704728
:1095A800E0240020024B03EBC00090F83E00704717
:1095B800E0240020024A0B2303FB00231971F1E584
:1095C800E0240020024A0B2303FB00235971E9E53C
:1095D800E0240020024A0B2303FB0023D971E1E5B4
:1095E800E0240020024A0B2303FB00239971D9E5EC
:1095F800E0240020024A0B2303FB00231972D1E563
:10960800E0240020024A0B2303FB00235972C9E51A
:10961800E0240020024A0B2303FB00239972C1E5D2
:10962800E0240020024A0B2303FB00231973B9E549
:10963800E0240020024A0B2303FB00235973B1E501
:10964800E0240020024A0B2303FB00239973A9E5B9
:10965800E0240020024A0B2303FB00200079704716
:10966800E0240020024A0B2303FB002040797047C6
:10967800E0240020024A0B2303FB0020C079704736
:10968800E0240020024A0B2303FB00208079704766
:10969800E0240020024A0B2303FB0020007A7047D5
:1096A800E0240020024A0B2303FB0020407A704785
:1096B800E0240020024A0B2303FB0020807A704735
:1096C800E0240020024A0B2303FB0020007B7047A4
:1096D800E0240020024A0B2303FB0020407B704754
:1096E800E0240020024A0B2303FB0020807B704704
:1096F800E0240020034B00EB8002134483F82C1075
:1097080062E600BFE0240020034B00EB8002134414
:1097180083F82D1058E600BFE0240020034B00EB2F
:109728008002134483F82E104EE600BFE024002088
:10973800034B00EB8002134483F82F1044E600BF6C
:10974800E0240020034B00EB8002134483F8301020
:109758003AE600BFE0240020034B00EB80001844E9
:1097680090F82C00704700BFE0240020034B00EB6A
:109778008000184490F82D00704700BFE0240020B6
:10978800034B00EB8000184490F82E00704700BF90
:10979800E0240020034B00EB8000184490F82F00D1
:1097A800704700BFE0240020034B00EB8000184402
:1097B80090F83000704700BFE0240020034B00EB16
:1097C8004002134483F82410AEE500BFE0240020D3
:1097D800034B00EB4002134483F82510A4E500BFB7
:1097E800E0240020034B00EB4002134483F82610CA
:1097F8009AE500BFE0240020034B00EB400018442A
:1098080090F82400704700BFE0240020034B00EBD1
:109818004000184490F92500704700BFE02400205C
:10982800034B00EB4000184490F82600704700BF37
:10983800E0240020024B03EBC003197636E500BF95
:10984800E0240020024B03EBC00359762EE500BF4D
:10985800E0240020024B03EBC003997626E500BF05
:10986800E0240020024B03EBC003D9761EE500BFBD
:10987800E0240020024B03EBC003197716E500BF74
:10988800E0240020024B03EBC00359770EE500BF2C
:10989800E0240020024B03EBC003997706E500BFE4
:1098A800E024002010B5054B03EBC0030446D9772C
:1098B800FFF7FCFC2046BDE8104035E5E024002019
:1098C800024B03EBC000007E704700BFE02400207D
:1098D800024B03EBC000407E704700BFE02400202D
:1098E800024B03EBC000807E704700BFE0240020DD
:1098F800024B03EBC000C07E704700BFE02400208D
:10990800024B03EBC000007F704700BFE02400203B
:10991800024B03EBC000407F704700BFE0240020EB
:10992800024B03EBC000807F704700BFE02400209B
:10993800024B03EBC000C07F704700BFE02400204B
:109948002DE9F0472C4CDDF82080099F1E4623188E
:10995800054693F844308A469146042B23D8DFE81D
:1099680003F003161B202500FFF71CFC63190122D6
:1099780004EBC50583F84420AB7F012B28D018D30E
:10998800022B2BD00FB123683B70BDE8F087FFF79F
:109998008DFC63190222EBE7FFF716FD631903221A
:1099A800E6E7FFF7C1FC63190022E1E7FFF75AFD7C
:1099B800F9E7BAF1000F03D023689B0C8AF800304E
:1099C800B9F1000FDED023689B0A89F80030D9E787
:1099D800002ED7D023689B0A3360D3E71EB12368D3
:1099E800DB0B5B013360B8F1000FCBD02368C3F306
:1099F800842388F80030C5E7E02400202DE9F843E7
:109A0800089E099D8146884617461C4600F076F850
:109A180080B96C21484600F0BEF8154B03EBC9032A
:109A28009B7F012B14D007D3022B16D005B12870C9
:109A3800BDE8F8836E21EDE7B8F1000F02D0830C82
:109A480088F80030002FF1D0C0F389233B80EDE780
:109A5800002CEBD0830A2360E8E714B1C30B5B0149
:109A68002360002EE2D0C0F384233370DEE700BF0A
:109A7800E0240020054A0B2303FB0023DA7A1AB9F5
:109A88000122DA72FFF78EBB704700BFE024002086
:109A9800054A0B2303FB0023DA7A1AB10022DA7293
:109AA800FFF780BB704700BFE0240020024A0B2369
:109AB80003FB0020C07A7047E0240020062808D85D
:109AC800DFE800F004080B0E111417000A4B1B689E
:109AD8000B607047084B1B6CFAE7074B5B69F7E7AD
:109AE800054B5B6BF4E7044B9B6AF1E7024B1B6A7F
:109AF800EEE7014BDB7AEBE7E0240020034B53F859
:109B08002000431E58425841704700BF28250020B6
:109B1800F8B541F080011746012000221E469DF845
:109B280018509DF81C40FFF77BF9394600220120A8
:109B3800FFF776F9314600220120FFF771F929462F
:109B480000220120FFF76CF9012221461046BDE8EA
:109B5800F840FFF765B910B541F0800114460120BF
:109B68000022FFF75DF92116002289B20120FFF7D4
:109B780057F9210C00220120FFF752F9C4F30F21F5
:109B880000220120FFF74CF90122E1B21046BDE89E
:109B98001040FFF745B910B5002201200C46FFF729
:109BA8003FF9002211460120FFF73AF90022114639
:109BB8000120FFF735F9002211460120FFF730F99F
:109BC800012200211046FFF72BF92146002201202F
:109BD800FFF726F9002211460120FFF721F900229C
:109BE800114604020120FFF71BF900221146044325
:109BF8000120FFF715F92402012204430021104631
:109C0800FFF70EF92402204310BD70B504460D4637
:109C18001646FFF7C0FF294640EA06022046BDE87F
:109C28007040FFF798BF70B504460D461646FFF71B
:109C3800B2FF294620EA06022046BDE87040FFF739
:109C48008ABF2DE9F8439DF8209098460F460646AE
:109C580014460025FFF79FFFC144414601234945AB
:109C68000BD304FA08F444402C4080EA0402394635
:109C78003046BDE8F843FFF76EBF03FA01F215431B
:109C88000131ECE710B50C2104464FF0FF32FFF725
:109C980062FF20460E21BDE81040FFF77CBF10B5DB
:109CA800CA4304460C21FFF756FF20460E21BDE8A3
:109CB8001040FFF770BF10B5074B012204461A5435
:109CC80020210022FFF747FF204600222421BDE87B
:109CD8001040FFF740BF00BF712E002013B57F2151
:109CE8000020FFF758FF5F4C00214FF4805220609E
:109CF8000846FFF730FF23685B4C012B0CBF0A2294
:109D08008A2204210020FFF726FF032205210020D4
:109D1800FFF721FF042220210020FFF71CFF00226B
:109D280010463721FFF717FF002210462121FFF7C1
:109D380012FF4FF4480224210020FFF70CFF4FF4D4
:109D4800483228210020FFF706FF4FF44832292126
:109D58000020FFF700FFA37DA27A0193637A0093A6
:109D6800002318460621FFF7D3FEA38A3F4A404C3A
:109D78005A4315210020FFF7EEFE6268602100209B
:109D8800FFF7E9FEA26861210020FFF7E4FEE389FE
:109D9800227B1C2143EA02420020FFF7DCFE2269F5
:109DA80059210020FFF7D7FE226A5A210020FFF729
:109DB800D2FE626A5B210020FFF7CDFEA26A94F80A
:109DC8002C30D1B2C2F30722009200220191104632
:109DD8005D21FFF79DFE226B5E210020FFF7BBFE91
:109DE800A26918210020FFF7B6FEE26919210020B8
:109DF800FFF7B1FE626B5C210020FFF7ACFEA26B9F
:109E08005F210020FFF7A7FEE26B52210020FFF739
:109E1800A2FE94F84030626C019394F841300093AC
:109E28006321D3B20020C2F30722FFF771FE94F832
:109E38004830002422462046019400947D21FFF7F3
:109E480067FE02212046FFF72AFF022220460D2145
:109E5800FFF7DBFE12212046FFF79DFE054B186039
:109E680002B010BD28250020902E002000710200AD
:109E7800D02E0020842E0020054B4FF080629A617E
:109E880000BF00BF00BF4FF480629A61704700BFF7
:109E980000040048000270478000704700127047B5
:109EA80080107047704700BF70B5044CA278637883
:109EB80042B1034B04221A7070BD00BF942F0020DA
:109EC80008300020FF2B00F22085DFE813F00001A6
:109ED8002C014701550164016F01740179017E016C
:109EE80087018F019801A101B501C901D801E201DB
:109EF800E701EC01F601FB0105020A021502200246
:109F08002B0236024D02540268021E051E051E056C
:109F180071027D02840299029E02A3021E051E059B
:109F28001E051E051E051E051E051E051E051E0511
:109F38001E051E051E051E051E051E051E051E0501
:109F48001E051E051E051E051E051E051E051E05F1
:109F58001E051E051E051E051E051E051E051E05E1
:109F68001E051E051E051E051E051E051E051E05D1
:109F78001E051E051E051E051E051E051E051E05C1
:109F88001E051E051E051E051E051E051E051E05B1
:109F98001E051E051E051E051E051E051E051E05A1
:109FA8001E051E051E05A802AD02B202B702BC02BC
:109FB800C102C602CB02D002D502DA02DF02E402F5
:109FC800E9021E05EE02F502FA02FF0204031E056D
:109FD80009031E050E031C03230329031E052E0374
:109FE80034033A031E051E051E051E051E051E0523
:109FF8001E051E051E051E051E051E051E051E0541
:10A008001E051E051E051E051E051E051E055804F7
:10A018005E0464046A0470047F048E049D04A3042F
:10A02800A904AF04B504BB04D104D704DD04E304D8
:10A03800E904EF04F504FB040005080511051705FC
:10A048001E051E051E051E051E051E051E051E05F0
:10A058003F0344034C03540359031E051E055E03C6
:10A0680063037D031E051E051E0581031E05860369
:10A078008B039B03A003A603AB03B003B5031E0524
:10A088001E051E05C5031E051E051E051E051E050B
:10A098001E051E051E051E051E05CB03D203D9038A
:10A0A800E003E703EE03F5031E051E051E051E0566
:10A0B8001E051E051E051E051E051E051E051E0580
:10A0C8001E05FC0343041E0549044E0453040020E6
:10A0D80003F02CFC9C4D9D4E3721B8B9A078FFF7B2
:10A0E8005AFDA37856F8233058436860984B1B787C
:10A0F8005BB1954B5A68974B1A60974B002A40F012
:10A1080009841A6842F008021A6070BDA078FFF747
:10A1180042FDA278914B53F82230C01A56F82230EB
:10A1280058436860E2E78E4B874D1878874E2121A7
:10A1380038B9FFF730FDA37856F8233058436860E4
:10A14800D4E70020FFF727FDA278844B53F822308C
:10A15800C01A56F8223058436860C7E77B4D24215F
:10A1680000206E68FFF717FDB047A37855F8233035
:10A178005843754B5860B9E7744D222100206E682A
:10A18800FFF709FD0002B047A37855F8233058437C
:10A198006D4B5860AAE76D4D6B68A8689847A3781F
:10A1A80055F823305843684B58609FE76D4B9A6ABF
:10A1B800654B5A609AE76B4B5A7A634B5A6095E73E
:10A1C800684B9A7A604B5A6090E70F210020FFF79E
:10A1D800E2FC5D4B00F00100586087E74FF09043C8
:10A1E800594A1B8A03F0010353607FE70F210020BF
:10A1F800FFF7D1FC544BC0F30020586076E70F21DD
:10A208000020FFF7C8FC504BC0F3C01058606DE742
:10A2180001210020FFF7BFFC810741BF4A4A53686C
:10A2280043F00103536002077FF560AF464A536865
:10A2380043F00203536059E701210020FFF7ABFC0C
:10A24800C30741BF404A536843F0010353604607C0
:10A258007FF54CAF3C4A536843F00203536045E72F
:10A26800FEF758F838B1A2783E4B03EB8213DA7D3B
:10A27800354B5A603AE7344B03221A7036E7334BB2
:10A28800252100205C68FFF786FCA0472E4B58600C
:10A298002CE7344B1A6B2C4B5A6027E7314BDA6AA0
:10A2A800294B5A6022E7294B272100205C68FFF7D9
:10A2B80072FCA047244B586018E72A4B5A6B224B74
:10A2C8005A6013E7214B262100205C68FFF763FCE6
:10A2D800A0471D4B586009E7224B9A6B1A4B5A60EE
:10A2E80004E7FEF717F80028C5D02D21A078FFF75E
:10A2F80052FC154B5860F9E6FEF70CF80028BAD066
:10A308002E21A078FFF747FC0F4B5860EEE6FEF7CA
:10A3180001F80028AFD02F21A078FFF73CFC0A4BAA
:10A328005860E3E6FDF7F6FF0028A4D03021A078B6
:10A33800FFF731FC044B5860D8E633210020FFF7C3
:10A348002AFC014B5860D1E6083000202C2500205B
:10A3580003300020F42F00209C2F00205C2E0020CA
:10A36800D02E0020902E002034210020FFF713FC6F
:10A378008B4B5860BAE601210020FFF70CFC45061C
:10A3880041BF874A536843F00103536004067FF5D1
:10A39800ADAE834A536843F002035360A6E6012139
:10A3A8000020FFF7F8FB7E4BC0F3012058609DE6C4
:10A3B80001210020FFF7EFFB10F0100F784B14BFBE
:10A3C800012200225A6091E601210020FFF7E3FBF9
:10A3D80010F0200FF2E7002003F0A8FA704D3221A8
:10A3E80020B9A078FFF7D7FB68607FE6A078FFF771
:10A3F800D2FBA2786B4B53F82230C01A686075E61E
:10A40800694B1A68664B5A6070E6684B1A78644B59
:10A418005A606BE6664B1A68614B5A6066E6654B94
:10A428005A685F4B5A6061E6624B9A685C4B5A60A7
:10A438005CE6604B1A7B5A4B5A6057E65D4BDA89EB
:10A44800574B5A6052E65B4B1A69554B5A604DE6BA
:10A45800584B1A7D524B5A6048E6564B5A7D504B22
:10A468005A6043E6534B1A6A4D4B5A603EE6514BCD
:10A478005A6A4B4B5A6039E64E4B9A6A484B5A60B7
:10A4880034E64C4BDA6A464B5A602FE6494B1A6B56
:10A49800434B5A602AE6474B9A69414B5A6025E676
:10A4A800444BDA693E4B5A6020E67C210020FFF7D6
:10A4B80072FB3B4B586019E63E4B5A6B384B5A605F
:10A4C80014E63C4B9A6B364B5A600FE6394B9A7D33
:10A4D800334B5A600AE6384B1A7B314B5A6005E613
:10A4E800344B1A782E4B5A6000E6344B2C4CD86902
:10A4F80018B905F0B3F96060F8E566210020FFF7A8
:10A508004AFB6060F2E565210020FFF744FB244B1D
:10A518005860EBE5002003F009FA214B5860E5E5A7
:10A52800244BDA6B1E4B5A60E0E5224B93F840202F
:10A538001B4B5A60DAE51F4B93F84120184B5A60C1
:10A54800D4E51C4B5A6C164B5A60CFE51B4B1A7A54
:10A55800134B5A60CAE5194A174B10685B6898474D
:10A568000F4B5860C2E5154A134B50685B68984713
:10A578000B4B5860BAE5124B1A68094B5A60B5E59F
:10A58800104B1A68064B5A60B0E50C4B9A7D044B89
:10A598005A60ABE5094B9A7E014B5A60A6E500BFAD
:10A5A80008300020742E0020642E0020922F0020F6
:10A5B8004C2E0020D02E00202C250020902E00208C
:10A5C800542E00201C2F0020A14BC8225A608DE574
:10A5D800A04B1A689E4B5A6088E59F4B1A789C4B93
:10A5E8005A6083E550210020FFF7D5FAA2789B4BEB
:10A5F80053F82230C01A9A4B53F822305843944BE0
:10A60800586073E5974BDA69914B5A606EE5954B44
:10A6180093F83C208E4B5A6068E5924B1A6A8C4B33
:10A628005A6063E58F4B5A6A894B5A605EE58D4BD9
:10A638009A8A874B5A6059E58A4B854C93F83D00B6
:10A6480018B904F02BFE606050E5002004F026FEE7
:10A65800C0F58040606049E5002004F023FE7C4B93
:10A66800586043E50021084604F027FE784B5860FF
:10A678003CE50121002004F020FE754B586035E5CB
:10A688000221002004F019FE714B58602EE50321C9
:10A69800002004F012FE6E4B586027E504210020CC
:10A6A80004F00BFE6A4B586020E50521002004F0F9
:10A6B80004FE674B586019E50621002004F0FDFDF3
:10A6C800634B586012E5624D00236B60FDF7F4FFA1
:10A6D8002871FDF7FCFF4FF0904368711B8AD8077B
:10A6E80048BFAB79A07848BF43F001034FF00F0192
:10A6F80048BFAB71FFF74FFAC10542BFAB7943F0D2
:10A708000203AB71020648BFAB79064648BF43F067
:10A718000403A07848BFAB71FEF71AF818B1AB79FB
:10A7280043F00803AB71F30748BFAB79A07848BF83
:10A7380043F010034FF0220148BFAB71FFF72BFA2B
:10A7480018B1AB7943F02003AB71A378424AD35CCC
:10A75800EB71CBE4434B93F83D203D4B5A60C5E485
:10A76800414B1A683A4B5A60C0E43E4B5A7E384B0C
:10A778005A60BBE43B4B1A7E354B5A60B6E4002066
:10A78800FEF708FF324B5860B0E40020FEF70AFFDE
:10A798002F4B5860AAE40020FEF75CFF2C4B586052
:10A7A800A4E40020FEF75EFF294B58609EE40020D9
:10A7B800FEF758FF264D20B9A078FEF763FF6860C2
:10A7C80094E4A078FEF77EFF68608FE40020FEF72F
:10A7D80049FF1F4D20B9A078FEF75CFF686085E44B
:10A7E800A078FEF77FFF686080E40020FEF73AFF5C
:10A7F800174D20B9A078FEF755FF686076E4A07879
:10A80800FEF768FF686071E40020FEF753FF104B05
:10A8180058606BE40020FEF79FFF0D4B586065E41D
:10A828000020FEF7A3FF0A4B58605FE40020FEF704
:10A83800A7FF074B586059E40020FEF7ABFF044B15
:10A84800586053E4094B5A79014B5A604EE400BFF3
:10A85800083000207C2E00208E2E0020742E002030
:10A868002C250020902E0020842E0020682E002009
:10A878000020FEF7C1FF2A4B586037E40020FEF79E
:10A88800C5FF274B586031E40020FFF719F8244B27
:10A8980058602BE40020FFF71BF8214B586025E493
:10A8A8000020FFF71DF81E4B58601FE40020FFF73B
:10A8B8001FF81B4B586019E40020FFF729F8184BC4
:10A8C800586013E4174B1A78154B5A600EE4164A71
:10A8D800164B10695B689847114B586006E4144A98
:10A8E800124B10685B6898470D4B5860FFF7FEBB2A
:10A8F8000F4B1A790A4B5A60FFF7F8BB0020FEF796
:10A90800B9FE074B5860FFF7F1BB054B03221A70DD
:10A91800FFF7ECBB1A6822F00802FFF7F5BB00BF8F
:10A9280008300020602E0020902E00202C250020CA
:10A93800682E002038B5B14A9378022B144600F0EF
:10A948001181032B00F01581002B40F0888153788A
:10A958004D2B00F0BC8039D8452B00F08A8018D8E0
:10A96800422B7CD006D8402B6DD0412B72D00322CD
:10A97800A34B66E0432B77D0442BF8D1A149D2F8FA
:10A98800033041F81C3F04221C20BDE83840FEF784
:10A99800CFBA482B7AD00BD8462B6FD0472BE6D1AD
:10A9A8009849D2F8033041F8083F04220820ECE720
:10A9B8004B2B7CD000F28680492BD8D1D278914B92
:10A9C800002A6FD1DA75D97D17203FE0552B00F0AA
:10A9D800A7801DD8512B00F0868008D84F2B7BD03C
:10A9E800502BC4D1874BD178997516202EE0532B64
:10A9F80000F08E8040F28480D2F80330012B00F200
:10AA08002E818049D37801F81A3F01221A20BCE729
:10AA1800832B00F098800BD8572B00F08D805C2B8F
:10AA2800A5D17849D37801F8273F01222720ACE740
:10AA3800852B00F09280C0F08B80FF2B97D1D278C5
:10AA4800714B1A7038BDD17840F2FF70BDE83840BC
:10AA5800FEF759BA6B4BD17819700020F6E7694BAD
:10AA6800D17859700120F1E7664BD178197104202B
:10AA7800ECE7644BD17859710520E7E76149D2F8D2
:10AA8800033041F80C3F04220C207EE75D49D3785F
:10AA980001F8243F01222420FEF74AFABDE8384095
:10AAA80002F00EBF56490122DA754A608BE7554C11
:10AAB800D178E1700320FEF726FAE078BDE8384047
:10AAC800FEF77AB84F4BD17899700220BEE74D4B0C
:10AAD800D17859751520B9E7D2F80310494BC9B296
:10AAE80059761920B2E7474D2A7DD20704D5E37875
:10AAF800DB0701D4FEF78EFAE17829751420A5E763
:10AB08004049D2F8033041F8203F042220203CE796
:10AB18003C49D2F8033041F8103F0422102034E7B2
:10AB2800D2F80330012B00F29A803649D37801F825
:10AB38001B3F01221B2028E73249D37801F8253F23
:10AB48000122252021E7D2F80320304B1A6138BDB5
:10AB58002F4BD2F803201A6038BDD2F803202B4BB4
:10AB68005A6138BD51782B4BD2F8032043F8212085
:10AB780038BD5378272B5DD017D8022B34D00CD88A
:10AB88004BB3012B7FF4F3AE234BD2F803205A606A
:10AB9800FDF790FB1D4BD86138BD1B2B3ED01C2BFD
:10ABA80042D0092B7FF4E3AE38BD2B2B48D007D811
:10ABB800292BD2F80320184B40D0D1D9DA6138BDFF
:10ABC8002D2B47D041D32E2B7FF4D1AE124BD2F888
:10ABD8000320DA6238BD104BD2F803201A60FDF763
:10ABE80069FB0A4B986138BD0B4BD2F803209A6079
:10ABF800FDF760FB054B186238BD00BF942F00209D
:10AC08000830002004000020023000202C250020FD
:10AC18000430002014300020202F0020D2F8033008
:10AC2800104ADBB2137338BDD2F803300D4ADBB2D9
:10AC3800537338BDD2F803200A4B87E79A6138BDB1
:10AC4800084BD2F803201A6238BD064BD2F803200D
:10AC58005A6238BD034BD2F803209A6238BD0422E9
:10AC680086E600BF202F0020554A00232DE9F04139
:10AC78001360544A544C1360544A63621360544A34
:10AC8800A36284F82C3084F82D3084F82E3004F137
:10AC980030014FF0FF301D4641F82300D5540133F1
:10ACA8002F2BF9D124210020FEF775FF494BA06016
:10ACB8001D70494D2B7E002B52D1484BC4F8EC3007
:10ACC8006360C4F8F030C4F8F43028210020D4F8C8
:10ACD800F460FEF760FFB0472921A8620020D4F88D
:10ACE800F460FEF758FFB0472A21E8620020D4F844
:10ACF800F460FEF750FFB0472B2128630020D4F8FA
:10AD0800F460FEF748FFB0472C2168630020D4F8B0
:10AD1800F460FEF740FFB04795F83D30A8634BBBA1
:10AD280001232F4A236000231946174642F82310AF
:10AD38000133B3F5807FF9D12A4EB27EEAB9F37EAA
:10AD48005BB3337903F0EF02012A34D1012384F88D
:10AD5800F830737D03B1012384F8F930BDE8F08140
:10AD6800214BC4F8EC30214B6360214BC4F8F03020
:10AD7800204BA8E74FF0FF33D3E7DFF87C804FF490
:10AD8800C365A5F214612846042241440435FEF740
:10AD980019F9B5F5CD6FF4D1D1E74FF4A765A5F54D
:10ADA800A7612846042239440435FEF70BF9B5F5A6
:10ADB800C36FF4D1C5E7212BC8D00023C7E700BF74
:10ADC800F42F0020103000202C2500209C2F00207C
:10ADD800622F0020712E0020902E0020AD9E0008CA
:10ADE80014300020040000209D9E0008A59E000845
:10ADF800A19E0008A99E0008A02F0020014B93F8EF
:10AE0800FA0070472C250020F8B5654E654A870181
:10AE1800F5190446A96A91420CD8EB6A934209D8FD
:10AE28002B6B934206D86B6B934203D8AB6B934260
:10AE380040F281803E44022200212046FEF7E5FED2
:10AE4800D6ED0A7AF8EE677A17EE900A08F02AFE2D
:10AE58000022554B08F07AFE4FA3D3E9002308F0EF
:10AE68009FFF09F085F8282102462046FEF773FE69
:10AE7800D6ED0B7AF8EE677A17EE900A08F012FE14
:10AE88000022494B08F062FE43A3D3E9002308F0EF
:10AE980087FF09F06DF8292102462046FEF75BFE80
:10AEA800D6ED0C7AF8EE677A17EE900A08F0FAFDFC
:10AEB80000223D4B08F04AFE37A3D3E9002308F0EF
:10AEC8006FFF09F055F82A2102462046FEF743FE97
:10AED800D6ED0D7AF8EE677A17EE900A08F0E2FDE3
:10AEE8000022314B08F032FE2BA3D3E9002308F0EF
:10AEF80057FF09F03DF82B2102462046FEF72BFEAE
:10AF0800B06B07EE900AF8EE677A17EE900A08F031
:10AF1800C9FD0022244B08F019FE1FA3D3E9002322
:10AF280008F03EFF09F024F802462C212046BDE82F
:10AF3800F840FEF710BE1D4E06EB840602220021E3
:10AF4800FEF771FED6F8F030A86A98472821024625
:10AF58002046FEF700FED6F8F030E86A9847292127
:10AF680002462046FEF7F7FDD6F8F030286B9847E2
:10AF78002A2102462046FEF7EEFDD6F8F030686B2F
:10AF880098472B2102462046FEF7E5FDD6F8F0301B
:10AF9800A86B9847C8E700BF000000A2941AED42CA
:10AFA800902E0020FFFF3F00000040422C2500208B
:10AFB80073B5034CA278637822B1042200F010BC68
:10AFC800942F0020FF2B00F25F85DFE813F00001CB
:10AFD80016013D014D01590175017F0196015D057D
:10AFE8005D055D055D05A101B301C401D401DD0165
:10AFF800E201E701F001F501FE0103020D0216026C
:10B008001F0228022C02300242025D055D055D0523
:10B018004F025D026B028802900294025D055D0595
:10B028005D055D055D055D055D055D055D055D0508
:10B038005D055D055D055D055D055D055D055D05F8
:10B048005D055D055D055D055D055D055D055D05E8
:10B058005D055D055D055D055D055D055D055D05D8
:10B068005D055D055D055D055D055D055D055D05C8
:10B078005D055D055D055D055D055D055D055D05B8
:10B088005D055D055D055D055D055D055D055D05A8
:10B098005D055D055D055D055D055D055D055D0598
:10B0A8005D055D055D059902A802B702D302E302BA
:10B0B800E902F60207030D03130321032D033303EB
:10B0C80039035D055D053F0345034B0356035D05E5
:10B0D8005F035D055D055D055D0569035D056F033E
:10B0E800790387035D055D055D055D055D055D0506
:10B0F8005D055D055D055D055D055D055D055D0538
:10B108005D055D055D055D055D055D055D05700415
:10B11800790482048B049404A704BA04CD04D604E9
:10B12800DF04E804F104FA04080511051A052305EB
:10B138002C0535055D055D053E0547054F0554059C
:10B148005D055D055D055D055D055D055D055D05E7
:10B158008E0393039C035D055D055D055D05A503F1
:10B16800AF035D055D055D055D055D055D055D0577
:10B17800B303E9030B04100416041B045D055D0505
:10B188005D055D055D055D055D055D055D055D05A7
:10B198005D055D055D055D055D055D055D055D0597
:10B1A8005D055D055D055D055D055D055D055D0587
:10B1B8005D055D055D055D055D055D055D055D0577
:10B1C8005D055D0523043204350443045104B94B7D
:10B1D800D4F803201878B84B38B91B6837215A437C
:10B1E80002B0BDE87040FEF7B6BC1968B34B1B68E7
:10B1F80001FB023237210020F2E7AE4BAE4D187842
:10B2080028B9D4F803302A6821215A43E8E72121D4
:10B218000020FEF7C0FCA378D4F8032055F82310CB
:10B2280001FB1200A54A502142F823001846FEF7F8
:10B23800B2FCA278D4F8033055F8221001FB1300B1
:10B248009F4B43F822004FE09E4B9B4DD4F80300E0
:10B2580001221A70D5F8EC309847A37855F82320C6
:10B26800242142431846BBE7934DD4F80300D5F890
:10B27800EC309847A37855F8232022214243F1E780
:10B288008D4DD4F80300D5F8EC3098470028B8BFA6
:10B298004042A8602021A078FEF77DFC400723D516
:10B2A800A678D4F8030005EB8605D5F8EC30984766
:10B2B80024210246304693E7834BD4F803209A6250
:10B2C800002002B0BDE87040FFF79EBD794B7E4874
:10B2D8001B78E17841724BB9827A807D01900091A8
:10B2E80018460621FEF714FC02B070BDC9080020FC
:10B2F80002B0BDE87040FEF775BA6E4B72491B7814
:10B30800E2788A72002BEFD1887D0190497AE6E7CE
:10B3180001210020FEF73FFCD4F8033020F00A0298
:10B32800D90748BF42F002029E0701D542F0080241
:10B33800012157E001210020FEF72DFCD4F803304D
:10B3480020F00502DD0748BF42F001029807EFD55B
:10B3580042F00402ECE7FCF7DDFF002800F09483DC
:10B36800D4F80320012A3FF628AEA178564B03EB08
:10B378008113DA75B8E7504BD4F80300D3F8EC30F2
:10B3880098472521024636E74F4BD4F803201A6325
:10B3980096E74D4BD4F80320DA6291E7464BD4F890
:10B3A8000300D3F8EC3098472721024623E7464BA1
:10B3B800D4F803205A6383E73F4BD4F80300D3F84B
:10B3C800EC3098472621024615E73F4BD4F8032076
:10B3D8009A6375E7FCF79EFF002800F05583D4F8C0
:10B3E80003202D21A078FBE6FCF794FF002800F04D
:10B3F8004B83D4F803202E21F4E7FCF78BFF0028B9
:10B4080000F04283D4F803202F21EBE7FCF782FFFA
:10B41800002800F03983D4F803203021E2E7D4F87B
:10B4280003203321E7E6D4F803203421E3E60121A1
:10B438000020FEF7B0FBD4F8033020F0C002D90793
:10B4480048BF42F040029B077FF572AF42F080028E
:10B458006EE701210020FEF79EFBD4F803301B02A3
:10B4680020F4407203F440731A4361E7012100207D
:10B47800FEF791FBD4F8033020F01002002B3FF4C4
:10B4880057AF42F0100253E701210020FEF783FB7B
:10B49800D4F8033020F02002002B3FF449AF42F0EB
:10B4A800200245E7002002F041FA78B9D4F80320D9
:10B4B800322197E7D02E00202C2500205C2E00207A
:10B4C800742E0020712E0020902E0020A078AB4B07
:10B4D800D4F8032053F8203032211A4480E6D4F8F7
:10B4E8000330002BFFF669ADA54A1360FCE6E2784D
:10B4F800A44B1A70F8E6D4F80320A34B1A60F3E6BD
:10B50800A24BD4F803005860A14BDD6925B903F0BC
:10B51800FDFE2A46602165E7024660216BE69B4BEB
:10B52800D4F8030098609A4BDD6925B903F000FF51
:10B538002A46612156E7024661215CE6934BD4F81E
:10B5480003001873924BDB694BB903F009FF1C2108
:10B55800A078FEF720FBC0F308021C2142E71C215B
:10B568000020FEF718FBD4F80320C0F3080040EAD7
:10B578000242F2E7854BD4F80320DA811C2100202F
:10B58800FEF709FBD4F8033000F47F02C3F3080385
:10B598001A43E2E77D4BD4F803201A6159212AE6C1
:10B5A8007A4AD4F803101378C9B21175002B3FF406
:10B5B8009BAE937D0191527D0BE07449D4F8032032
:10B5C8000B78D2B24A75002B3FF48EAE8B7D097D85
:10B5D8000191009206210022002083E66B4BD4F8EB
:10B5E80003201A625A2106E6684BD4F803205A62EF
:10B5F8005B2100E6D4F80320644BD1B29A62C2F30F
:10B60800072293F82C300191009200225D21E3E794
:10B618005E4AD4F80330D362926AD1B2C2F30722E9
:10B6280001910092DBB2F0E7584BD4F803201A637B
:10B638005E21E0E5554BD4F803209A611821DAE53C
:10B64800524BD4F80320DA611921D4E54F4BD4F8D2
:10B6580003205A635C21CEE54C4BD4F803209A634F
:10B668005F21C8E5494AD4F803301178DBB29375F5
:10B6780000293FF439AE117D9CE7D4F80330022B42
:10B688003FF69BAC434BE2781A732DE6D4F80330AF
:10B698003E4A012B0ABF404900230B70137023E672
:10B6A8003A4BD4F80320DA635221A4E5374BE1780A
:10B6B8005A6C83F84010019193F84130009308E0E8
:10B6C800324BE17883F841105A6C93F840308DE89A
:10B6D8000A00D3B26321C2F307227DE72B4BD4F8CB
:10B6E80003205A6493F84010E5E7294BD4F8032067
:10B6F8001A72F9E5274BD4F80300D3F8EC309847D1
:10B70800234B1860F0E5234BD4F80300D3F8EC3052
:10B7180098471F4B5860E7E51C4B1D491B78E0789C
:10B728008875002B7FF4E0AD8A7AEEE5184BE27855
:10B738009A76D9E550210020FEF72DFA154DA37809
:10B74800D4F8032055F8231001FB12000B4A0F49C7
:10B7580042F823004C225A438A5C002A3FF4C4ADC5
:10B7680021211846FEF717FAA278D4F8033055F8C5
:10B77800221001FB1300094B63E500BF742E002063
:10B78800642E0020922F00204C2E0020D02E002066
:10B79800902E00202C250020712E00205C2E0020E9
:10B7A800BA4DD4F80320E9698A423FF49DADB84BFD
:10B7B8001878A0B9002A0FDD012003F0E3FDD4F8C2
:10B7C8000320A0785421FEF7C6F9A378D4F8032003
:10B7D80005EB8313DA6187E503F0D4FDF5E706226C
:10B7E800AC4B86E6A94BE27883F83C207CE5A74B76
:10B7F800D4F803201A625321FDE4A44BD4F80320A3
:10B808005A6271E5A14AD4F803309382A24A1521FD
:10B818005A43F0E4D4F80300A04B9C4A012118B91C
:10B8280082F83D0019605FE582F83D104FF0FF3265
:10B8380064E6E2789A4B5CE69A4BD4F803201A60E7
:10B84800002002F02FF800287FF44EADD4F8032032
:10B858001221C7E5D4F803300F2B3FF6AEABE178E1
:10B868008A4B0020597602B0BDE8704002F077BDDF
:10B87800D4F803307BB1012B7FF49FAB834A137656
:10B88800864B894AC3F8EC20884A5A60884AC3F82C
:10B89800F020884A08E07D4A1376804B864AC3F830
:10B8A800EC205A60C3F8F020C3F8F4201CE5D4F863
:10B8B80003100020C9B202B0BDE87040FDF74EBECB
:10B8C800D4F803100020C9B202B0BDE87040FDF7FB
:10B8D80051BED4F803100020C9B202B0BDE87040D0
:10B8E800FDF768BED4F803100020C9B202B0BDE865
:10B8F8007040FDF767BE0020FDF7B4FED4F80310D2
:10B90800C9B228B9A07802B0BDE87040FDF76ABE98
:10B91800A07802B0BDE87040FDF784BE0020FDF7B6
:10B92800A1FED4F80310C9B228B9A07802B0BDE8C6
:10B938007040FDF75FBEA07802B0BDE87040FDF72B
:10B9480081BE0020FDF78EFED4F80310C9B228B9D5
:10B95800A07802B0BDE87040FDF754BEA07802B0F0
:10B96800BDE87040FDF766BED4F803100020C9B2E8
:10B9780002B0BDE87040FDF74DBED4F803100020BA
:10B98800C9B202B0BDE87040FDF7B4BED4F80310E8
:10B998000020C9B202B0BDE87040FDF7B5BED4F8CA
:10B9A80003100020C9B202B0BDE87040FDF7B6BE72
:10B9B800D4F803100020C9B202B0BDE87040FDF70A
:10B9C800B7BED4F803100020C9B2FDF7BBFEA278B9
:10B9D8003A4B03EBC203D4F803205A7184E4D4F839
:10B9E80003100020C9B202B0BDE87040FDF7E6BE02
:10B9F800D4F80310002049B202B0BDE87040FDF74A
:10BA0800E7BED4F803100020C9B202B0BDE8704008
:10BA1800FDF710BFD4F803100020C9B202B0BDE88A
:10BA28007040FDF70FBFD4F803100020C9B202B070
:10BA3800BDE87040FDF70EBFD4F803100020C9B26E
:10BA480002B0BDE87040FDF70DBF144BD4F80300F9
:10BA5800D3F8EC3098470D4B186145E40F4BD4F8F8
:10BA68000300D3F8EC309847144B4AE6134BD4F84C
:10BA780003201A7138E4D4F803100020C9B202B0C8
:10BA8800BDE87040FDF7A6BD0322A9E6902E002070
:10BA9800D02E002008300020007102002C25002044
:10BAA800502F0020842E00209D9E0008A59E00088F
:10BAB800A19E0008A99E0008AD9E0008682E0020DF
:10BAC8002DE9F341B94CBA4D2378D4F803006B70D3
:10BAD8006422222B2A70686001F04B8000F2B48047
:10BAE8000F2B00F00B8554D8072B00F05B8314D87C
:10BAF800032B00F0E48108D8012B00F04081022BD1
:10BB080000F09C8102232B7042E1052B00F0478353
:10BB180040F2EB81FEF7C8F93AE10B2B00F07D8487
:10BB280028D8092B00F06E8340F25483A378022BA7
:10BB380000F00684032B00F00884002B40F0658495
:10BB480063789C4A502B00F0D38300F27983462B0C
:10BB580000F0C18300F25E83422B00F0B68300F24E
:10BB68005483402B00F09883412B00F0AB830323D0
:10BB78002B7096E30D2B00F0778440F26384A37852
:10BB8800002B00F09C84022B00F0A28404232B706D
:10BB9800FEE0192B00F0D2852ED8152B00F02D854C
:10BBA80018D8132B00F0DF84142BABD1824B834AB7
:10BBB80019681368884280F2108523F0030343F064
:10BBC800040313601368002940F0128543F008034A
:10BBD8001360DDE0172B7A4B00F0A28540F29D85BB
:10BBE8009A6A002A00F0D480013A9A6203EB820232
:10BBF800D2F8FC205A62CBE01E2B00F0B5860CD898
:10BC08001B2B00F0BD85C0F0AA851C2B7FF47AAFF2
:10BC18006B4B002283F8F920BAE0202B00F01D8737
:10BC280040F2DD866278644B0A2A00F25D87DFE81D
:10BC380012F0560765076A076F0775077D078207C1
:10BC480087078C0791079507812B01F034803DD831
:10BC5800412B01F0188020D8252B00F0D38711D86C
:10BC6800232B00F08E87242B7FF44CAF6378052BB1
:10BC780000F28E80DFE813F08D0794079B07A20778
:10BC8800A907B007272B00F0EF87C0F0C587402B26
:10BC98007FF438AF01F05CFD7AE0452B00F0FF87B8
:10BCA80007D8432B00F0F78740F2F18701F0D3FD66
:10BCB8006EE0472B00F0FB87C0F0F587802B7FF400
:10BCC80021AF3F4B002283F8F92061E0892B01F076
:10BCD800CE802AD8852B01F0308014D8832B01F030
:10BCE800088041F20080334B1B7D9B0701F12180C6
:10BCF800B0F55B7F80F09F80314B042283F8F920F8
:10BD0800C3F8440144E0872B01F08480294B41F2B9
:10BD18001A806278012A01F06380C1F04F80022AFC
:10BD280001F0678003232B7032E08D2B01F018811E
:10BD38000ED88B2B01F0CC8041F2B1806678002EB2
:10BD480001F0CC80012E01F0D98003232B701FE075
:10BD5800F22B01F09781FF2B01F0D381992B7FF40F
:10BD6800D1AE6378072B01F28981DFE813F0480927
:10BD7800500955095A095F0975097D098209A3788F
:10BD8800002B58D1002001F08DFDD8B106232B706F
:10BD9800084B93F827302BB194F90030002BA4BF3F
:10BDA80063782B7002B0BDE8F08100BF942F0020AB
:10BDB8000830002004000020F42F00209C2F0020D1
:10BDC8002C250020A078BC4B01264FF0006231469C
:10BDD8001E54FDF71AFFA078B84B03EB8013DB7DE8
:10BDE8003BBB32462021FDF7B6FEA678B44BD4F80B
:10BDF800032053F8260003EB86035043D3F8EC30B6
:10BE08009847242102463046FDF7A5FEA0784FF05A
:10BE180080520721FDF7F9FEA0784FF00062072154
:10BE2800FDF701FF4FF000620121A078FDF7FBFE4E
:10BE3800AEE70222D6E704232B70A9E7A0780028F2
:10BE4800F9D101F02FFD0028A0D1A0789A4B012646
:10BE58004FF0006231461E54FDF7D7FEA078974B8D
:10BE680003EB8013DB7D43BB32462021FDF773FED5
:10BE7800A678934BD4F8032053F8260003EB8603E7
:10BE88005242D3F8EC3050439847242102463046BA
:10BE9800FDF761FEA0784FF080520721FDF7B5FE4F
:10BEA800A0784FF000620721FDF7BDFE4FF0006259
:10BEB8000121A078FDF7B7FE6AE70222D5E7A3784B
:10BEC800002BB8D17C4901220A707C49C87D40B951
:10BED8002021FDF740FE00222421A078FDF73BFE3B
:10BEE80056E7022220211846F3E7A0780028A2D1BD
:10BEF80001F0D8FC00287FF449AF6178012900F0EF
:10BF08008A803FD302297FF443AFA3781E0640F10D
:10BF1800FC80D9077FF53CAF684BDB7D002B40F0F8
:10BF2800E6800522644F664E2021FDF714FE3B781B
:10BF380033B1B26824210020FDF70DFE00233B70C9
:10BF48004FF0805207210020FDF76DFE4FF0006290
:10BF580000200721FDF759FE5A4BD4F80320187822
:10BF6800594B002840F0C58053F8223032683721F9
:10BF78005A43FDF7F0FD4FF0006201210020FDF764
:10BF880052FE05E7A0784FF000620121FDF73DFE63
:10BF9800A0784A4B03EB8013DB7D93BB052220215D
:10BFA800FDF7D9FD444FA078454E3B5C43B106EB05
:10BFB800800324219A68FDF7CEFDA3780022FA5465
:10BFC8004FF080520721A078FDF72DFE4FF0006258
:10BFD800A0780721FDF719FEA0783A4A4C2343437D
:10BFE800D25CD4F8033072B956F820205A4337216E
:10BFF800FDF7B1FD4FF000620121A078FDF713FEB7
:10C00800C6E60622CBE7314A56F8201052F820201F
:10C0180001FB0322EBE7A0784FF00062FDF7F5FD86
:10C02800A078264B03EB8013DB7D73B90522202112
:10C03800FDF791FD224FA0783A18127B012A38D0DB
:10C0480005D3022A44D000260BE00622EFE7372169
:10C05800FDF7A1FDA378D4F8036057F8233003FB5C
:10C068000606A078DFF8508018F800304BB107EBCF
:10C07800800324219A68FDF76EFDA378002208F852
:10C088000320A0784FF080520721FDF7CCFDA0785F
:10C098004FF000620721FDF7B8FD3246A07837213E
:10C0A800FDF759FD4FF000620121A078FDF7BBFDB7
:10C0B8006EE62121CCE700BF712E0020902E0020D3
:10C0C8002C250020D02E0020A02F00205C2E002040
:10C0D8005021FDF760FDA378A74957F8232051F8B0
:10C0E8002330D4F80360C01A02FB0606B9E706221B
:10C0F80018E753F82220A078A04B316853F8203075
:10C10800002001FB0232372133E79D4A02EB8312FC
:10C11800D27D002A37D1052218462021FDF71BFDC4
:10C12800984FA078984E3B5C43B106EB80032421DE
:10C138009A68FDF710FDA3780022FA544FF0805258
:10C148000721A078FDF76FFD4FF000620721A07866
:10C15800FDF75BFDA0788D4A4C234343D15CD4F8AE
:10C1680003308B4A034481B952F8233056F8202013
:10C178005A433721FDF7EFFC4FF000620121A07808
:10C18800FDF751FD04E60622C6E752F823207B4B53
:10C1980056F8201053F8203001FB0232E9E7FEF789
:10C1A80007FFF5E5A378002B7FF445AE6378C92B2C
:10C1B80004D0D22B08D003232B70E9E5012275495E
:10C1C8005A20FCF7B5FEE3E5042273495C20FCF72E
:10C1D800AFFEDDE5A378002B7FF42DAE6378C92B85
:10C1E80004D0D22B08D003232B70D1E50122694952
:10C1F8005A20FCF7E7FECBE5042267495C20FCF7F0
:10C20800E1FEC5E5FEF796FBC2E5442B61D05ED999
:10C21800537958E04B2B65D00AD8482B5FD05CD3B4
:10C22800492B7FF4A4ACD37D003318BF01234AE027
:10C238004D2B5BD058D34F2B7FF499AC537E42E003
:10C248005C2B5FD012D8532B56D006D8512B51D027
:10C25800522B7FF48CAC136A35E0552B50D04DD35C
:10C26800572B7FF484AC92F825302CE0832B56D0E2
:10C2780009D8812B49D04FD8802B7FF478AC424B1A
:10C2880093F8F9301FE0852B4FD04BD3FF2B7FF469
:10C298006EAC424B1B78C7E740F2FF70FCF778FEA4
:10C2A80068603F4B1B78002B3FF472AD3D4B6A68CA
:10C2B8001A603D4B002A40F0AB801A6842F0080231
:10C2C8001A6065E513786B60EBE75378FBE7137941
:10C2D800F9E7D369F7E7D368F5E79368F3E792F8E6
:10C2E8002430F0E7D378EEE79378ECE7537DEAE77C
:10C2F800937DE8E7137DE6E71369E4E7937EE2E7D9
:10C30800D37EE0E792F82730DDE71F4B93F8F9304A
:10C318001A1F53425341D6E71B4B5B6AD3E71A4BAC
:10C328001B69D0E7214B1B68CDE7174A20485369A2
:10C3380043F2390100FB0313536123F00043C2E7C2
:10C3480062781C4B53F82230BDE76378282B4ED017
:10C3580034D8022B48D007D8002B43D0012B7FF4C8
:10C3680006AC154B5B68AEE7092B9AD0272B7FF4F8
:10C37800FEAB114BD4E700BF742E00205C2E0020CA
:10C38800902E0020712E00202C250020D02E002079
:10C39800A02F0020AA2E0020AC2E00200230002062
:10C3A80003300020F42F00209C2F002004300020B0
:10C3B8006D4EC64114300020202F00202B2B1CD09E
:10C3C80007D8292B16D02A2B7FF4D1AB964BDB69E3
:10C3D80079E72D2B16D013D32E2B7FF4C8AB924BB5
:10C3E800DB6A70E7904B9EE78F4B9B686BE78E4B41
:10C3F8005B6968E78C4B9B6965E78B4B1B6A62E757
:10C40800894B8AE7884B9B6A5DE70423FFF7B0BB3B
:10C418001A6822F008021A60BAE4A378022B0ED137
:10C428006078372808D800F5A77080498000042272
:10C438000144FCF77DFDABE403232B70A8E404233F
:10C448002B70A5E4A378022B0BD160783728F3D89A
:10C4580000F5A7707549800004220144FCF7B2FD7D
:10C4680096E404232B7093E4A378002B7FF4E3ACC9
:10C478006378012B09D004D3022B0AD003232B7035
:10C4880086E4002002F0D6FA82E4002002F0DAFA0C
:10C498007EE4002002F0DEFA654B68601B78002B12
:10C4A8003FF476AC634B1860634B1A6818B942F0D6
:10C4B80008021A606CE422F008021A6068E4FBF7CC
:10C4C80040FF0028B8D0D4F80300FCF70FF95FE468
:10C4D8006378072B08D818B91846FCF773F857E49F
:10C4E8001846FCF78FF853E4FF2BA5D1431C0ABF6D
:10C4F800504BC0B21878FCF7A5F849E4A378012B93
:10C5080024D004D3022B25D004232B700AE06078B2
:10C51800082803D8FCF7A7F8686003E00A2810D1B8
:10C5280000236B60424B1B78002B3FF431AC414B2E
:10C538006A681A60404B8AB91A6842F008021A60A1
:10C5480026E4FF28EED1FCF7B7F8E5E7607803F0BA
:10C558005FFAE1E76078FCF797F8DDE71A6822F000
:10C5680008021A6014E46278324B092A26D8DFE8F8
:10C5780002F005090C0F13191C1F22071A68104432
:10C5880018601BE01A68101AFAE71A685043F7E7B0
:10C598001A6892FBF0F0F3E7196891FBF0F200FBE0
:10C5A8001210EDE71A681040EAE71A681043E7E747
:10C5B8001A685040E4E71A68D2431A601A681E4B9A
:10C5C8002AB91A6842F008021A60FFF7E1BB1A6834
:10C5D80022F008021A60FFF7DBBB0BBF23F006034B
:10C5E80023F0050343F0010343F00203FFF7E9BA20
:10C5F80023F008031360FFF7CBBB63780C2B3FF6DF
:10C60800C7ABDFE803F0071D262F38414B545D66A2
:10C618006F788100084B1B681F077FF5B9AB074B84
:10C628005862FFF7B5BB00BF202F0020DC2A00208E
:10C6380003300020F42F00209C2F00202C25002000
:10C64800AE4B1B681E073FF5A3ABAD4B5862FFF717
:10C658009FBBAA4B1B68D9077FF59AABA84B5862BA
:10C66800FFF796BBA54B1B68DA073FF591ABA44BC8
:10C678005862FFF78DBBA14B1B685B077FF588AB42
:10C688009F4B5862FFF784BB9C4B1B6813F0050F48
:10C698003FF47EAB9A4B5862FFF77ABB974B1B6807
:10C6A8009F077FF575AB964B5862FFF771BB934BAD
:10C6B8001B689E073FF46CAB914B5862FFF768BB51
:10C6C8008E4B1B68D9067FF563AB8D4B5862FFF71D
:10C6D8005FBB8A4B1B689A067FF55AAB884B58623A
:10C6E800FFF756BB854B1B685B067FF551AB844B48
:10C6F8005862FFF74DBB814B1B681F067FF548AB9F
:10C708007F4B5862FFF744BB7C4B1B68DE057FF507
:10C718003FAB7B4B5862FFF73BBB5862FFF738BB18
:10C728009A6A072A3FF634AB511C03EB82029962DE
:10C73800596AC2F8FC105862FFF72ABB63782E2B9F
:10C7480004D8704A0121D154FFF722BBFF2B7FF494
:10C7580073AE6B4B012283F82D20FFF719BB63786A
:10C768002E2B04D8674A0021D154FFF711BBFF2BA9
:10C778007FF462AE624B002283F82D20FFF708BBDE
:10C788005F4E96F82C309BB9411C04BF5E4A106876
:10C798004FF00A030BBF43435843C6F81C31C6F891
:10C7A8001C01FBF787FD0123C6F8200186F82C3011
:10C7B8006378042B3FF6ECAADFE803F0034472A881
:10C7C8001900FBF777FDD6F82031C01A0028D6F8F3
:10C7D8001C31B8BF4042984295BF736A002303F1E9
:10C7E800FF3386F82C3098BF7362FFF7D1BAA07870
:10C7F80002F030F940B9414A86F82C00136823F05A
:10C8080010031360FFF7C4BAD6F81C31ABB1FBF7BD
:10C8180051FDD6F82031C01A0028D6F81C31B8BF0F
:10C828004042984209D9354A002386F82C301368CB
:10C8380043F010031360FFF7ABBA736A013B7362EE
:10C84800FFF7A6BA0F21A078FDF7A5F910F00107A8
:10C8580009D02A4A002386F82C30136823F01003E5
:10C868001360FFF795BAD6F81C31A3B1FBF722FD88
:10C87800D6F82031C01A0028D6F81C31B8BF40427B
:10C88800984208D91D4A86F82C70136843F01003A3
:10C898001360FFF77DBA736A013B7362FFF778BADA
:10C8A8000F21A078FDF777F910F0800709D0134A17
:10C8B800002386F82C30136823F010031360FFF769
:10C8C80067BAD6F81C31A3B1FBF7F4FCD6F82031CF
:10C8D800C01A0028D6F81C31B8BF4042984208D97F
:10C8E800064A86F82C70136843F010031360FFF7AC
:10C8F8004FBA736A013B7362FFF74ABA9C2F002054
:10C908002C250020622F0020F42F00200F21A07872
:10C91800FDF741F910F4807709D0B34A002386F86F
:10C928002C30136823F010031360FFF731BAD6F8E0
:10C938001C31A3B1FBF7BEFCD6F82031C01A002881
:10C94800D6F81C31B8BF4042984208D9A64A86F8A2
:10C958002C70136843F010031360FFF719BA736A59
:10C96800013B7362FFF714BA6378142B3FF664AD8A
:10C97800A278AAB99D4A9E49927E41F82300002ACE
:10C988003FF406AA002B3FF403AA03F285108000A7
:10C99800A0F2146304221944FCF7CAFAFFF7F8B9A5
:10C9A800FF2A7FF448AA924F73B94FF4C366A6F2E0
:10C9B80014613046042239440436FCF7B9FAB6F556
:10C9C800CD6FF4D1FFF7E4B903F285108000A0F22F
:10C9D800146104223944FCF7ABFAFFF7D9B960783F
:10C9E80014283FF629ADA378C3B9814B53F820200A
:10C9F800804B6A601B78002B3FF4CAA97E4B1A60F3
:10CA0800794B2AB91A6842F008021A60FFF7C0B9D0
:10CA18001A6822F008021A60FFF7BAB9FF2B7FF4F0
:10CA28000AAA734F70B94FF4C366A6F21461304670
:10CA3800042239440436FCF7C5FAB6F5CD6FF4D1B3
:10CA4800FFF7A6B900F285108000A0F21461042255
:10CA58003944FCF7B7FAFFF79BB96678142E3FF60E
:10CA6800EBACA078614F10F0800F1AD0C20706D542
:10CA780021210020FDF78FF85D4B43F82600BB7E8F
:10CA8800002B3FF485A9607800283FF481A900F2C3
:10CA980085105A49800004220144FCF749FAFFF73F
:10CAA80077B900287FF4C7A92121FDF774F8504908
:10CAB800BB7E41F82600002B3FF46AA96378002B5F
:10CAC8003FF466A9A0781E1803F2851318440422BF
:10CAD80001EB86018000FCF72BFAFFF759B94849AA
:10CAE8001A6809680A441A601A683F4B002A3AD142
:10CAF8001A6842F008021A60FFF74AB940491A68F2
:10CB08000968521AEFE73E4A196812684A43EAE789
:10CB18003B491A68096892FBF1F2E4E7384A186859
:10CB2800116890FBF1F201FB1202DCE734491A6844
:10CB380009680A40D7E732491A6809680A43D2E700
:10CB48002F491A6809684A40CDE72D490A68D24337
:10CB58000A60C9E719682A4A1160C5E7284A1968AE
:10CB680010681860F8E71A6822F008021A60FFF7E0
:10CB78000FB9214B1B68C4F80330FEF719FAFFF709
:10CB880007B91D4B1B68C4F80330FDF7D3FEFFF748
:10CB9800FFB8154A136803F00F031360FFF7F8B8DE
:10CBA800114A136823F010031360FFF7F1B80E4A17
:10CBB800136823F020031360FFF7EAB80A4A1368E2
:10CBC80023F040031360FFF7E3B8074A136823F024
:10CBD80080031360FFF7DCB8034A136823F48073FB
:10CBE8001360FFF7D5B800BF9C2F00200400002079
:10CBF800A02F002003300020F42F00208C290020D3
:10CC08001030002062782E2A3FF616ACC34B03EB97
:10CC180082031863FFF7BCB8C04BC14AD3F824118C
:10CC28001160C04AD3F828111160D3F82C215A6238
:10CC3800BD4AD3F830111160D3F8342183F82C2081
:10CC4800D3F83821C3F82021D3F83C21C3F81C219C
:10CC5800B64993F84021885C08B101208854002225
:10CC680083F82E20FFF794B8A378002B7FF4E3A86D
:10CC78006378142B3FF6E0ABA94A1168AC4A42F836
:10CC88002310FFF785B800F087FDFFF781B800F0A3
:10CC9800C5FDFFF77DB800F0DDFDFFF779B800F0BE
:10CCA800DBFDFFF775B800F0D8FDFFF771B800F0AD
:10CCB800D5FDFFF76DB863782BB1012B09D003239D
:10CCC8002B70FFF765B8954B012283F8F920FFF721
:10CCD8005FB8B0F55B7FBFF4AEA8904A82F8F93030
:10CCE8005062FFF755B88D4B022283F8F920FFF701
:10CCF8004FB88A4A8D48002382F82D3082F82E30AA
:10CD080002F130064FF0FF37194646F82370C15438
:10CD180001332F2BF9D1824B82F8F9101960814B1E
:10CD280051621960804B916282F82C101960FFF7EC
:10CD38002FB808232B70FFF72BB8784B002283F805
:10CD4800F920FFF725B87B4A7B4E01271770B0F50D
:10CD58005B7F9A78327027D21B7D13EA070823D1AC
:10CD68006946FCF750F99DF8003073709DF8013062
:10CD7800B3709DF80230F3709DF8063033719DF85A
:10CD8800053073719DF80430B3719DF80330F37169
:10CD980086F808803B46F15C327A01330A44082B56
:10CDA8003272F8D1FEF7F4BF3B460022F254013349
:10CDB800082BFBD133783372FEF7EABF5D4A9B78C4
:10CDC800012111705C4A13705C4B1968002301390A
:10CDD800013311F8010FD054082BF9D1FEF7D8BF51
:10CDE8000523EB715A23AB7123236A712B71FEF76C
:10CDF800CFBF504A9B785248012111704E4A137098
:10CE0800002301331918082B11F8091CD154F8D143
:10CE1800FEF7BEBF6378032B3EF6BAAFDFE803F038
:10CE280002101D223D4B93F8F920EA7193F82C204B
:10CE3800D3F84431AA711A0A6A712B71FEF7A8BF98
:10CE4800364B93F8F920EA7193F82C205B6AAA71A3
:10CE58001A0A6A712B71FEF79BBF314B1B686B6016
:10CE6800FEF796BF2F4B1B686B60FEF791BF637888
:10CE7800002B7EF48DAFA17800297EF489AF40F2B3
:10CE8800D24398427EF484AF40F2FF70FCF73BF83F
:10CE9800FCF7C0F80120FBF72CFCFEF779BF62789D
:10CEA800284B9AB91A70284AE37813701B4A92F8EB
:10CEB8004811264A1170264900220A7025490A702D
:10CEC800254A11780B431370FEF762BF0122E9E788
:10CED800124B012283F84921FEF75ABF0422694602
:10CEE80040F2FB70FCF76EF8009BD4F803209A42DE
:10CEF80006BF01236B606E60FEF74ABFA3782A2B3A
:10CF080007D10422154940F2FB70FCF711F8FEF72F
:10CF18003FBF03232B70FEF73BBF00BF2C2500202B
:10CF2800F42F0020103000209C2F0020622F0020BA
:10CF3800A02F0020F82F0020F92F0020000000204B
:10CF480000800008582E0020782E00205E2F002038
:10CF5800722E0020932F0020592E0020972F00209A
:10CF68006378032B47D8DFE803F01B0234426A4E8C
:10CF7800D6F84C11002206F5A8738A423EF408AF91
:10CF880053F82270874202F1010720D103EB87038F
:10CF9800043B01398A4214D3C6F84C11FEF7F8BE97
:10CFA8005D4BD3F84C21092A9DBF511CC3F84C1185
:10CFB80003EB8203092394BFC3F850012B70FEF7DB
:10CFC800E7BE53F8040F43F8040C0132E2E73A468F
:10CFD800D3E7514A0023C2F84C31194602F5A8722A
:10CFE80042F8231001330A2BFAD1FEF7D1BE0A23E7
:10CFF8006B60FEF7CDBE03232B70FEF7C9BE474B0F
:10D0080098427EF418AF02F009FCFEF7C1BE02F0A8
:10D018000DFC6860FEF7BCBE02F014FC6860FEF709
:10D02800B7BE02F015FC6860FEF7B2BEB0F5005F4F
:10D03800BEF601AF400080B202F005F80004686057
:10D04800D4F803004000013080B201F0FCFF6B68A7
:10D0580018436860FEF79CBE304B98427EF4EBAEF6
:10D0680001F0D2FFFEF794BE02F024F96860FEF7E3
:10D078008FBE02F005FC6860FEF78ABE03232B70A2
:10D08800FEF786BE6378812B7EF482AEA378922B5E
:10D098007EF47EAEA379A32B7EF47AAE6379B42BAB
:10D0A8007EF476AE2379C52B7EF472AEE378D62B68
:10D0B8007EF46EAE1A4B4FF400629A6172B6FBF7BB
:10D0C80025FB184B184800261E60314603F07BFAF2
:10D0D8003146164803F077FA134803F0CFF913489E
:10D0E80003F0CCF94FF0A04002F054FE104802F0D3
:10D0F80051FE104805F087FB3046FBF7FAFAFEF7B9
:10D1080047BE40F2D24398427EF442AE024B01221F
:10D1180083F87821FEF73CBE2C2500204E61BC0028
:10D128000004004810E000E05800024058040240A3
:10D138000004005000040040F7B50F4C07460E46A7
:10D1480094E803008DE803000C49C1F803300C4B48
:10D158008A7000220F704E701A70FEF7B1FC094AEF
:10D16800217882F8FA109DE80300636884E80300D8
:10D17800184603B0F0BD00BF08300020942F0020EF
:10D18800033000202C250020F7B504461F4A637899
:10D198001370A3785370E37893702379937163794C
:10D1A8005371A3791A4D1371E379D3700E4695E83C
:10D1B8000300184B00221A708DE80300FEF780FC6C
:10D1C800154B1A786F462B469AB9327072702A78C6
:10D1D800B2706A78F270EA793271AA7972716A79F2
:10D1E800B2712A79F27197E8030083E8030003B06B
:10D1F800F0BD012AF7D10948721EF11D10F8014F40
:10D2080002F8014F8A42F9D1EDE700BF942F0020C0
:10D218000830002003300020F82F0020F92F0020CC
:10D228002DE9F743274B284C1B7813B994F879312B
:10D238006BB1264B1B78063BDBB2192B04D8244A6A
:10D2480022FA03F3D90702D4002384F8483194F86A
:10D258004831204E032B40F0D3813378002B3FD147
:10D26800DFF878801C4F98F8020098F801503B7856
:10D2780005441D447B781D44FB791D44BB791D443E
:10D288007B791D443B791D44FBF75EFC98F801004F
:10D29800FBF75AFC3878FBF757FC7878FBF754FC17
:10D2A800F879FBF751FCB879FBF74EFC7879FBF776
:10D2B8004BFC3879EDB2FBF747FC2846FBF744FCFA
:10D2C80018E000BF023000202C250020942F0020F9
:10D2D80011020002F82F002008300020040000206E
:10D2E800012B07D1B54F0025785D0135FBF72CFCE4
:10D2F800092DF9D1B24B1A78984672B3B14BDFF8C1
:10D30800FC921B78032B23D1AF4F99F80030B878E3
:10D318007D7805440A351D44FBF716FC7878FBF741
:10D3280013FC8020FBF710FC8A20FBF70DFC002083
:10D33800FBF70AFC0020FBF707FC0020FBF704FCC6
:10D34800EDB299F80000FBF7FFFB2846FBF7FCFB62
:10D35800002389F8003088F80030002384F8483129
:10D36800337084F8793194F8783113B10120FBF7E0
:10D37800C0F994F849314BB194F8F830B3FA83F313
:10D388005B0984F8F830002384F849310DF107006F
:10D39800FBF7FAFB002800F06681FBF713FC10B1DD
:10D3A800002384F87A3194F87A219DF80710531CE9
:10D3B800DBB22244092B84F87A3182F87B1151D1EF
:10D3C800002384F87A31804B94F87B215978914274
:10D3D80005D093F82510002944D08A4242D193F809
:10D3E80025307A48934208BF01234FF0000208BF56
:10D3F80084F879311346115C01320B44082ADBB2F8
:10D40800F9D194F883219A4240F02981704B94F81D
:10D418007C211A7094F87D215A7094F87E219A70B4
:10D4280094F87F219A7194F880215A7194F8812197
:10D438001A7194F88221DA70FAF73CFF654B664A54
:10D44800186094F8F91000231370032284F8482117
:10D458004A1E012A84F87A31604A02D9052918BF80
:10D468000123137094F8F930042B04D1584B197820
:10D478000A0640F1238194F84821082A04D840F28A
:10D488005113D340DF0701D4FEF71AFB94F8483153
:10D49800092B6FD1FAF70EFFA369514DC01A002866
:10D4A8002A68B8BF4042904208D94E4B1A78012AE0
:10D4B80004BF02221A70FAF7FDFEA061FAF7FAFE1D
:10D4C800E3696A68C01A0028B8BF4042904208D988
:10D4D800444B5A78012A04BF02225A70FAF7EAFE2E
:10D4E800E061FAF7E7FE236AAA68C01A0028B8BF05
:10D4F8004042904208D93B4B9A78012A04BF022245
:10D508009A70FAF7D7FE206294F82D3093B394F806
:10D518002E307BBB334A34481D46D15C022940F08B
:10D52800C18050F823104E1C00F0BB802F4A84F8AD
:10D5380040311268C4F824212D4A1268C4F8282101
:10D54800626AC4F82C212B4A61621268C4F830213F
:10D5580094F82C20C4F834210023D4F82021C4F8EE
:10D56800382184F82C30D4F81C21C4F83C2101233C
:10D5780084F82E3094F84831092B06D194F8F92014
:10D58800022A04BF052284F8F920D4F84C21002A85
:10D5980000F09180092B40F08E8094F8F930012B2F
:10D5A80040F08980616A1448002350F823508D4266
:10D5B8007DD1052384F8F9307DE000BFF92F0020E4
:10D5C800932F00205E2F002004000020A7260020B3
:10D5D800942F0020582F00205D2F002003300020BA
:10D5E800202F0020622F00205C250020F42F00202F
:10D5F800103000209C2F00207C260020722E002056
:10D60800042B7FF477AE424FDFF81081B8787D782D
:10D61800002301220544154488F8013088F80020C9
:10D62800C8F80430FBF790FA7878FBF78DFA98F889
:10D638000000FBF789FA98F80100FBF785FA98F8DB
:10D648000700FBF781FA98F80600FBF77DFA98F8CF
:10D658000500FBF779FAEDB298F804002BE60423ED
:10D6680084F84831FEE694F8F930013B012B3FF687
:10D67800F9AE636AB3F55B7F0FD2FBF738F860B198
:10D68800606A2449431C6362FBF7BDFC092384F8E4
:10D698004831214B01221A70E4E6002384F8F9305E
:10D6A800E0E6D55401332F2B7FF437AF62E701331F
:10D6B8009A427FF47AAF03B0BDE8F08394F848014A
:10D6C800082804D840F25112C240D207F3D4D4F843
:10D6D8004401124DD3F803306970B0F55B7F6B607D
:10D6E80012D20C49FBF788FC0A49D4F84401FBF72D
:10D6F800B3FC38B1D4F844310133C4F8443165235C
:10D708002B70D8E70723FBE707232B70002351E78B
:10D7180004000020942F002003300020083000204F
:10D72800704710B5094CFAF7C5FD2368C01AB0F563
:10D73800FA7F09D94FF09042938A9BB283F008038D
:10D748009382FAF7B7FD206010BD00BFB026002015
:10D7580010B50F4B0F4C5A78042A15D8DFE802F0A1
:10D7680003070A0D1000FAF7BFFD606010BDFAF755
:10D77800CFFDFAE7FAF7CEFDF7E7FAF7E2FDF4E7AF
:10D788009878FCF7BBF9F0E70323237010BD00BFBE
:10D79800942F00200830002038B51D4B9C781D467A
:10D7A80094BB5A782AB1012A1A4D21D003232B7031
:10D7B80038BDD3F8030018B9BDE83840FAF7C5BF3B
:10D7C8001046FAF7C5FF70B15021A878FCF7E3F9C5
:10D7D800212102460446A878FCF7BDF922463721E4
:10D7E800A878FCF7B8F9A878BDE83840FAF7AABFD6
:10D7F8002046FAF7ADFF28B9074B9C8A84F40064E9
:10D80800C4F3C0246C6038BD024B04221A7038BDC2
:10D81800942F002008300020000400480B4A537859
:10D828002BB1012B0AD00A4B03221A707047D2F889
:10D83800030008B902F03CB80120FBE7D2F8030066
:10D8480008B902F02FB81846FBE700BF942F002054
:10D858000830002070477047704770470E4BDA78E1
:10D868004FF090434FF4801199610C4B42F40A42F7
:10D878009A811A89D107FCD59A8900229A81074B87
:10D888001A89D207FCD54FF09042102191619B89EB
:10D89800034A9BB253607047942F0020003C00401D
:10D8A80008300020054A135C02440033527818BF40
:10D8B80001230AB143F0020318467047B42600203A
:10D8C80010B5184B184C00201870587094F8243074
:10D8D800DA0704D513F0080317D0FAF793FE94F883
:10D8E8002430980705D5D9064FF0010011D5FAF76D
:10D8F80089FE94F824305A0712D59B064FF002008F
:10D908000AD5BDE81040FAF77DBE1846FAF75AFE68
:10D91800E5E7FAF757FEECE7BDE81040FAF752BE24
:10D9280010BD00BFB426002004000020034B18449B
:10D938008078431F58425841704700BFB4260020E2
:10D948002DE9F74FAA4CE57804F104084DB9E8B27F
:10D95800FAF789FE08F805000135082DF7D10123EB
:10D96800E370DFF8ACA2A34F272500264FF0020989
:10D97800F0B2FAF778FE18F80630834216D0331D55
:10D9880008F806005AF82330022B0AD0032B02D0DD
:10D99800012B0BD150B17B5D012B08BF07F8059017
:10D9A80004E018B97A5D012A00D17B550136082EAA
:10D9B80005F10105DCD1904FFB6993B18F4D2E78AD
:10D9C8007EB9FAF777FC8E4B1B68C01A0028FB69F2
:10D9D800B8BF4042984204D93046FCF76CF901239D
:10D9E8002B703B6A93B1874D2E787EB9FAF762FCAB
:10D9F800854B1B68C01A00283B6AB8BF4042984252
:10DA080004D93046FCF757F901232B702221207BDB
:10DA18007E4EFCF7C0F88046207BFCF733F90F21D7
:10DA28000546207BFCF7B7F88246207B06EB80137F
:10DA38001B6913B3002B88EAE872A2EBE872B8BF3F
:10DA48005B429A4219DD23185B7B43B94FF0806231
:10DA58000121FCF7DAF8237B012223445A73EA07F1
:10DA68001BD5207B634AC31CD15C012912D102213A
:10DA7800D1540121FCF713F90FE023185B7B002B2D
:10DA8800EDD04FF080620121FCF7CDF8237B002216
:10DA98002344E3E7D35C002BEBD0AB000CD5207B11
:10DAA800544A00F10F03D15C012904BF0221D1546B
:10DAB8004FF00051FCF7F3F8280507D5B8F1000F2F
:10DAC80004D14FF40061207BFCF7E9F8E90407D59D
:10DAD800B8F1000F04D14FF48051207BFCF7DFF838
:10DAE800AA0407D5B8F1000F04D14FF40051207BE8
:10DAF800FCF7D5F86B0407D5B8F1000F04D14FF443
:10DB08008041207BFCF7CBF8A8070BD5207B394A4E
:10DB180000F10903D15C012904BF0221D15402217B
:10DB2800FCF7BDF8237B01211AF08000A17304EBF8
:10DB3800030275D0D07B78B9D173354A1A44127B69
:10DB480012F0010F08D002211B2211FB0323294ADE
:10DB5800D05C012808BFD154237B1AF4807104EBF0
:10DB6800030267D0117C81B901211174284A1A4433
:10DB7800527B12F0010F08D00E331E4A12F8131010
:10DB8800012904BF022102F81310FAF793FB636915
:10DB9800C01A0028B8BF40420A2840F39F80207B63
:10DBA8001C4DFBF7ABFF02461B4B207B1B49002A91
:10DBB8004FD0A26901440544B2F57A7F4FF00002C4
:10DBC8000091019503EB800311463DD3FBF7B8FEA6
:10DBD8000023A361257B63199B78052B56D8DFE8C2
:10DBE80013F042006E01C90113022602710200BF40
:10DBF800B4260020622F0020040000205D2F0020A2
:10DC0800582F0020502E0020542F0020902E002046
:10DC1800202F00208E2E00207C2E0020602E002039
:10DC2800D17B002998D0D073C04A1A44127B12F0D5
:10DC3800020F87E7107C0028A7D01174BB4A1A444A
:10DC4800527B12F0020F96E7FBF7D8FEA369013367
:10DC5800BFE7014405440091019503EB8003114699
:10DC6800FBF7CCFEB6E74C236B43B14AD35C6BB1F0
:10DC7800284600F0EFFE48B906EB85132846597A86
:10DC8800C908FBF7AFFD25440123AB70207B00F0EA
:10DC9800D3FB207B06EB80135B7ED3B15021FBF7CF
:10DCA8007AFF237BDFF888E29D004C2101FB03E12A
:10DCB8006219C96B126AA2EB010E8645234403D888
:10DCC8000A44904240F24D82012283F824206319CD
:10DCD800186200232373FAF7EDFA6061257BC5B952
:10DCE800944B1A789B46A2B1B8F1000F4FF032015D
:10DCF8002846DFF85092C0F23882FBF74CFFD9F87B
:10DD08000020024432212846FBF725FF00238BF828
:10DD1800003097F92430002B80F22D824FF0904389
:10DD2800B3F8109009F0010997F82430DA072DD5D7
:10DD3800257B625D002A00F02382DFF80CB2B9F17E
:10DD4800000F03D194F82530012B03D01BF80530C0
:10DD5800DB071BD5002328466355FFF7A3FD30B921
:10DD6800754B122153F825202846FBF7F4FE227B39
:10DD78001BF8023023F001030BF8023097F8243027
:10DD8800180740F10E820020FAF73CFC97F824307F
:10DD98009A0712D5227B06EB821103F01003497E05
:10DDA800002940F002821AF0010F00F00482002BD3
:10DDB80000F004820120FAF705FC97F824305D078B
:10DDC80057D5257B63195B78002B00F0FB81DFF8C2
:10DDD8007881B9F1000F03D194F82530012B03D0D5
:10DDE80018F80530580744D54C23514E6B43F35C63
:10DDF80043B950212846FBF7CEFE2121024628468A
:10DE0800FBF7A9FE257B18F8053023F0040308F872
:10DE180005306319002228465A70FFF743FD30B9D0
:10DE2800454B122153F825202846FBF794FE207B0A
:10DE38004C234343F35C8BB1FAF78AFC70B1502151
:10DE4800207BFBF7A8FE212102460546207BFBF735
:10DE580082FE2A463721207BFBF77DFE207BFAF7DE
:10DE680071FC97F82430990640F125820220FAF7D0
:10DE7800C9FBBB7D84F82590002B00F06D8294F8D7
:10DE88002650002D00F02282012D00F02E822B4D0D
:10DE980094F826202978914200F05E82A37B002B1B
:10DEA80000F05A82BB7D012B40F03C82002A00F032
:10DEB8003F82207BFBF7FFFEFAF74DFC49E2002288
:10DEC80005212846FBF747FE194B4C2202FB053279
:10DED8002846117D937D0191527D009206210022F2
:10DEE800FBF716FE79212846FBF755FE7F282DDC27
:10DEF800C0F18009284604222021FBF72CFE104A95
:10DF080028462421FBF727FE21212846FBF743FE5C
:10DF1800372100EB09022846FBF71DFEFAF7CAF97C
:10DF280004EB85032544D8610223AEE6202F0020A8
:10DF3800D02E0020912F0020842E002044000020A5
:10DF480040420F004C2E0020502F0020B0F5C07F1B
:10DF580002DAC0F5C079CDE7B0F5207F02DAC0F566
:10DF68002079C7E7B0F5607FB4BFC0F56079C0F528
:10DF78009069BFE7FAF79EF904EB8503DB69C01ADD
:10DF88000028B8BF4042B0F57A7F7FF77FAE06EB36
:10DF98008513D3F81C90B9F1000F0BD02121284626
:10DFA800FBF7F9FD502102462846FBF7D4FD25442E
:10DFB80003236AE64A4620212846FBF7CCFD4A4659
:10DFC80024212846FBF7C7FD50212846FBF7E3FD2F
:10DFD800212102462846FBF7BEFD21212846FBF7F2
:10DFE800DAFD372102462846FBF7B5FD0422202139
:10DFF8002846FBF7B0FDC34A24212846FBF7ABFDB2
:10E00800C14B01225A55D2E728464FF0C05207218A
:10E01800FBF709FE2846BD4A0721FBF7F6FDFAF78C
:10E0280049F904EB85032544D86104232DE6FAF762
:10E0380041F904EB8503DB69C01A0028B8BF4042E8
:10E04800B0F57A7F7FF722AE4FF0194207212846B4
:10E05800FBF7E9FD06EB85135B7E0BB119072ED59F
:10E068004FF0206228460721FBF7CFFD2846802283
:10E078000521FBF770FD4FF0007228460121FBF7E0
:10E08800C4FD59212846FBF786FDA14A4C2303FB12
:10E098000523502118619F4B0022284643F825206C
:10E0A800FBF779FD212181462846FBF774FD9A4B41
:10E0B800A9EB000043F8250025440523E5E54FF0CA
:10E0C8000072CFE74C236B43914A12F803B0BBF1BF
:10E0D800000F7FF4DBAD06EB85194FF004620721D2
:10E0E8002846FBF7A0FD032205212846FBF733FD50
:10E0F80099F8163099F80A20019399F80930009395
:10E1080006215B462846FBF703FD1F212846FBF73F
:10E1180069FB631983F802B099F81730FBB901223B
:10E1280020212846FBF717FD002224212846FBF76B
:10E1380012FD21212846FBF72EFD764B53F82520AA
:10E148002121821A2846FBF706FD4FF000720121B3
:10E158002846FBF768FD6C4B01225A5596E50222CA
:10E16800DEE7002283F82420B3E5FBF714FDD9F895
:10E178000020821AC6E50020FAF775FA8146D3E531
:10E18800664B5B5D13F01A0F3FF400AE01231221BA
:10E1980028466355FBF7DFFC97F8243019077FF50D
:10E1A800F2AD0020FAF70EFAF0E5224492F82420A6
:10E1B800002A3FF4FCAD002B3FF4FCAD0120FAF738
:10E1C80021FAFAE5FAF7D6FA00283FF452AE207B96
:10E1D800FAF7BEFA00287FF44CAE207B06EB8013DA
:10E1E8001A6A9AB31AF4804F30D093F83C30012B56
:10E1F8001CD8FBF760FD207B454A4C234343D35C86
:10E208005BB15021FBF7C7FC237B434A52F823201C
:10E218002121821A1846FBF79EFC207B06EB80130F
:10E2280093F83C30012B01D1FAF78FFA207B2318A1
:10E2380001225A7012210022FBF78DFC97F8243036
:10E248009A064FF002003AD5FAF7BCF9207B06EBA4
:10E2580080135A6A002A3FF40CAEDB69304D8BBB41
:10E2680001F0FCFA237B06EB8312A0EB08000028E0
:10E27800516AB8BF404288427FF6FBAD92F83C2015
:10E28800012A02D81846FBF716FD207B06EB8016FC
:10E2980096F83C30012B01D1FAF757FA287B054450
:10E2A8000123002212216B70FBF755FC97F82430EC
:10E2B8009B067FF5DBAD0220FAF784F9D9E5FAF77A
:10E2C800A1F9C3E76621FBF766FCCBE70120FAF763
:10E2D800CAF9012806D1A36A642B10D9A56284F86B
:10E2E8002600D4E50023A362D1E52846FAF7BBF956
:10E2F8000028F7D1A36A642B01D9A062EFE70133A4
:10E30800F1E700BF40420F00712E0020000040815D
:10E31800D02E00205C2E0020742E00208E2E00208F
:10E32800B4260020022B7FF4C4AD012A7FF4C1ADCE
:10E338005021207BFBF72FFC212102460646207B3B
:10E34800FBF709FC32463721207BFBF704FCFAF780
:10E3580009FA94F826302B7003B0BDE8F08F38B571
:10E3680005460C46A1B9FBF716FC214620F4E072DD
:10E378002846FBF7F0FB4C236B431C4AD35C9BB34A
:10E3880028464FF000620721BDE83840FBF73DBC46
:10E398000021FBF700FC04F00303022B20F4E072D9
:10E3A8001CD0032B1DD0012B01D142F04002630782
:10E3B80048BF42F4807214F0080418BF42F4007297
:10E3C80000212846FBF7C7FB002CD9D128464FF07F
:10E3D80000620721BDE83840FBF725BC42F0800207
:10E3E800E5E742F0C002E2E738BD00BFD02E0020CA
:10E3F80038B5104B03EB80130446DB7D0D46B3B9EB
:10E4080001222021FBF7A7FB20464FF0805207216D
:10E41800FBF7FBFB20464FF000620721FBF703FCEC
:10E428002A4620462421BDE83840FBF794BB022247
:10E43800E7E700BF902E00202DE9F84FC44F0446AF
:10E448004FEA84190F21FBF7A6FB07EB0901020A23
:10E458000B7AD1F8048013F0400F1ABF02F0010BB9
:10E4680057F8092057F809A04FEAD01008BF00F064
:10E47800010B03F03F061DBF00F00100C2F1000AC6
:10E48800C8F1000802F0010013F0800F4FF090432C
:10E498001B8A18BFDB430A2E03F0010300F2B28186
:10E4A8000122B24012F4C06F40F01B8212F4F07FD8
:10E4B80040F0388112F01E0F00F0A481A54D2B5DAD
:10E4C800013B0E2B00F29E81DFE813F00F001E00C7
:10E4D8002D0039004900530062007100AF00E300CD
:10E4E800E9009C0124010202A20201212046FBF757
:10E4F80052FB05EB840301225860023E964B96427C
:10E508001A551AD8022332E005EB84035A6842F000
:10E51800020201212046FBF71EFB51462046FFF769
:10E5280067FF032323E0002800F06C8121212046A7
:10E53800FBF731FB894B43F82400042317E005EB74
:10E5480084035A6842F0010201212046FBF703FBCD
:10E55800CAF100012046FFF74BFF052307E0BBF196
:10E56800000F00F04F812046FBF7A5FB06232B5533
:10E5780048E105EB840301215A68204622F0030292
:10E58800FBF7E9FA41462046FFF732FF0723EEE79B
:10E59800BBF1000F40F0368159462046FFF728FFAF
:10E5A800C8F100012046FFF723FF0823DFE7BBF18E
:10E5B800000F00F0278121212046FBF7ECFA00210B
:10E5C80006462046FFF714FF644A52F824309B1B86
:10E5D80042F8243005EB84034F445A68012122F0A5
:10E5E80003022046FBF7B7FAFB7DE3B90522202199
:10E5F8002046FBF7B0FA424624212046FBF7ABFA47
:10E608004FF0805207212046FBF70DFB4FF00062C8
:10E6180007212046FBF7F9FA324637212046FBF757
:10E628009AFA0923A3E70622E1E70F212046FBF720
:10E63800B2FAC00740F1E68021212046FBF7ABFA89
:10E64800474B002118602046FFF7D2FE4C23634356
:10E65800444AD75C4FB93A4637212046FBF77BFA44
:10E668003A4621212046FBF776FA21212046FBF77E
:10E6780092FA3D4B502143F824002046FBF78BFAD1
:10E68800033E3A4B012E43F8240049D8C8F1000153
:10E69800CBE0BBF1000F00F0B5800B2367E7BBF1BF
:10E6A800000F40F0AF8021212046FBF774FA59464D
:10E6B80006462046FFF79CFE022396FBF3F605EB81
:10E6C80084034F445A68012122F003022046FBF7D5
:10E6D80042FAFB7DE3B9052220212046FBF73BFAED
:10E6E800424624212046FBF736FA4FF08052072194
:10E6F8002046FBF798FA4FF0006207212046FBF707
:10E7080084FA324637212046FBF725FA0D232EE7F7
:10E718000622E1E70F212046FBF73DFAC10771D534
:10E728000E2324E70B4D2A5D013A0E2A6AD8DFE84A
:10E7380012F01F002F0040004C005D0069006B00C4
:10E748006900690093009D0081003D01CF006F01C1
:10E75800902E0020E0260020712E0020542E00204C
:10E768001C2F0020D02E00205C2E0020742E0020AC
:10E77800AA4B012120461955FBF70DFA05EB840336
:10E78800062E58603FF4BEAE082E7FF4D6AEB9E62A
:10E79800062E05D105EB84035A6822F00302B6E67B
:10E7A800082E7FF4BAAE05EB84035A6822F0030200
:10E7B800AFE6721F012A05D820B1062E3FF4BDAE80
:10E7C8000F23D4E6F3B10C23D1E6052E05D105EBD2
:10E7D80084035A6822F00302B4E6072E7FF4B8AE29
:10E7E80005EB84035A6822F00302ADE6721F012A82
:10E7F80005D8BBF1000F02D0052EE1D182E6002B2F
:10E808007FF4C4AEBDE8F88F002BFBD1073E012E84
:10E818000AD905EB840301215A6822F0030242F069
:10E8280002022046FBF797F941462046FFF7E0FD34
:10E838000A239CE6002BE5D1073E012E7FF626AF82
:10E8480005EB840301215A6822F0030242F0010219
:10E858002046FBF780F919E7002BD3D02121204669
:10E86800FBF799F905EB8403986016E7002BC9D1EB
:10E8780021212046A600FBF78EF9AB194F445A68B0
:10E88800824622F0030201212046FBF764F9FB7D52
:10E89800E3B9052220212046FBF75DF942462421F1
:10E8A8002046FBF758F92E444FF0805207212046A6
:10E8B800FBF7B9F94FF0006207212046FBF7A5F9ED
:10E8C800B268924402229AFBF2F21BE70622E1E7C1
:10E8D80005EB840301215A682046FBF73CF9002325
:10E8E80045E64F4D2B5D013B0E2B8BD801A252F80C
:10E8F80023F000BF39E900080DE800080DE800081A
:10E908000DE800080DE800080DE800080DE800080B
:10E918000DE800080DE800085DE900080DE80008AA
:10E928000DE80008B5E90008E7E8000819EA00085A
:10E938003A4B01224FF4102120461A55FBF7AFF944
:10E9480040F6682207212046FBF75FF9092E7FF47D
:10E958009DAE69E70E212046FBF71DF9C2037FF53E
:10E9680051AF4F4400212046FFF742FDFB7DDBB944
:10E97800052220212046FBF7EEF8424624212046B6
:10E98800FBF7E9F84FF0805207212046FBF74BF9D7
:10E998004FF0006207212046FBF737F93621204661
:10E9A800FBF7F9F80246ADE60622E2E70F2120461A
:10E9B800FBF7F1F8C3077FF525AF0E232121204689
:10E9C8002B55FBF7E8F8174B002118602046FFF796
:10E9D8000FFD4C236343144AD55C4DB92A463721B1
:10E9E8002046FBF7B8F82A4621212046FBF7B3F862
:10E9F80021212046FBF7CFF80C4B502143F8240087
:10EA08002046FBF7C8F80A4B43F82400BDE8F88F06
:10EA180000212046FFF7ECFC82E600BF712E0020A3
:10EA2800E02600201C2F0020D02E00205C2E002085
:10EA3800742E0020024B1A5C0AB901221A5470473E
:10EA4800E0260020024B1A5C0AB10F221A547047C4
:10EA5800E0260020014B185C704700BFE02600202C
:10EA6800F8B599422DED028B04460D46164632DA6A
:10EA78005B1A07EE903A331B07EE103AF8EEE77A86
:10EA8800B8EEC77A274B87EE878A274693ED007A38
:10EA9800DFED257AB8EEC77A68EE277AF4EEC77A02
:10EAA800F1EE10FA44BFBDEEE77A17EE102A93EDA7
:10EAB800017A48BF1A60B8EEC77AF4EEC77AF1EE69
:10EAC80010FAC4BFFDEEE77AC3ED017AB74207DB5F
:10EAD800BDEC028BF8BDFBDDC1F580421344C8E7ED
:10EAE8003B1B07EE103A07EE905AB8EEC77AF8EEDD
:10EAF800E77AB8B2E8EE077A00F1806000F5E03016
:10EB08004000FDEEE77A013717EE901A4B42C3F347
:10EB18000D03C1F30D0158BF594289B201F07CFFC2
:10EB2800D4E700BFEC26002000007A4473B5F9F75B
:10EB3800C1FB0446F9F7BEFB001B0028B8BF4042E2
:10EB48006328F7DD4FF4E070FAF722FA044640F242
:10EB5800C110FAF71DFA05464FF4E170FAF718FAF2
:10EB6800064640F2C310FAF713FA210605D42A061E
:10EB780003D4330601D41F2803D9002006460546CE
:10EB88000446009033462A4621460020F9F722FE23
:10EB980002B070BD4FF090434FF480129A610D4B54
:10EBA8004FF426429A811A89D007FCD5988900210A
:10EBB80000049981074B20F07F421989C907FCD5C9
:10EBC8004FF0904110208861988980B21043800AE4
:10EBD800704700BF003C00400C4B002240211A72D5
:10EBE80010465972D9601A615A6103EB4201013229
:10EBF800402A0883F9D14FF480420549C3F8982088
:10EC08000A684968521AC3F89C207047EC2600200D
:10EC180048000020024B03EB4000008B00B2704715
:10EC2800EC260020684620F00701C74A8D4631B51A
:10EC380092F8A0001346002840F0CD8192F8A12058
:10EC4800002A43F6FF7218BF1146C04A107A0028FE
:10EC580000F0F880C3F8A410B3F8A81089B2C3F87C
:10EC6800AC105969D3F8A40001445961D3F8A41031
:10EC7800B1F5005F1969D3F8A4000144A8BFA1F554
:10EC880080411961197A0131C9B21972197A3F297B
:10EC980084BF00211972587AD968884280F2EB80C3
:10ECA800D3F8B010002940F0E680597A0131C9B292
:10ECB8005972197AD3F8A40003EB410100B2088312
:10ECC800D3F8A410B1F5805F05DBD3F8A410B1F533
:10ECD800405FC0F237811969587A91FBF0F1C3F8A7
:10ECE800B810D3F8B8100029BEBFD3F8B81001F592
:10ECF8008041C3F8B810D3F8B810D3F8B010013178
:10ED0800C3F8B010D3F8B010402947D1117A0029C0
:10ED180044D00021C3F8B010D3F8B810D3F8BC0021
:10ED2800091AC3F8C010D3F8C010B1F5005FD3F8C2
:10ED3800C01040F30F81A1F58041C3F8C010D3F88B
:10ED4800C010C3F8C410D3F8C010DFED816A0029E1
:10ED5800BEBFD3F8C0104942C3F8C01093ED307A53
:10ED6800B8EEC77AC6EE877AFDEEE77AC3ED037A86
:10ED7800D9684029C4BF4021D960D868D168884281
:10ED8800BCBFD168D960D3F8B810C3F8BC10D3F8A9
:10ED9800C4004FF474714143C3F8C810587A11691C
:10EDA800884280F21081D3F8C4505169D3F8984052
:10EDB800D3F8B800694391FBF4F10144C3F8CC10CF
:10EDC800D3F8C8005168884280F2CD805168D3F8E2
:10EDD800C8004942814280F2C6800022C3F8D02090
:10EDE800D3F8D020D3F8CC100A44C3F8CC20D3F8F9
:10EDF800CC205142C1F30D01C2F30D0258BF4A4263
:10EE0800C3F8CC20D3F8CC20002A05DAD3F8CC20DC
:10EE180002F58042C3F8CC205A7A402A40F0D680C6
:10EE2800D3F8CC20D3F8D410521A002AB8BF5242D3
:10EE3800022A00F3CB80D3F8D420C3F8CC20D3F82F
:10EE4800CC1089B293F8D82032B1B1F5804F3CBFCD
:10EE5800D3F8DC2032F81110A3F8A81093F8E020BA
:10EE68002AB193F8E020013AD2B283F8E020BDE855
:10EE7800314085467047197A587A091AC3F8B41090
:10EE8800D3F8B4100029BEBFD3F8B4104031C3F88A
:10EE9800B4105969D3F8B40003EB4000008B00B2FA
:10EEA800091A5961D3F8B41003EB4101098B09B26F
:10EEB800B1F5005F1969D3F8B40003EB4000008B8B
:10EEC80000B2A1EB0001A8BF01F580411961587A91
:10EED800D96888427FF7EDAED3F8B01089077FF480
:10EEE800E8AE597A0139C9B25972197A587A091AA9
:10EEF800C3F8B410D3F8B4100029BEBFD3F8B410C7
:10EF08004031C3F8B4105969D3F8B40003EB40009A
:10EF1800008B00B2091A5961D3F8B41003EB410110
:10EF2800098B09B2B1F5005F1969D3F8B40003EB96
:10EF38004000008B00B2A1EB0001A8BF01F58041A1
:10EF48001961B6E65969C7E6EC260020480000209A
:10EF58000000004311F5005FBFF6F1AED3F8C01012
:10EF680001F58041E9E6D3F8C8001168884201DD5F
:10EF7800926933E71168D3F8C8004942814202DD3B
:10EF8800926952422AE7D3F8C800516888420FDDD7
:10EF9800D3F8C800116888420ADAD3F8C810546850
:10EFA8009269D3F89C00091B4A4392FBF0F215E7DB
:10EFB8009069D3F8C8405268D3F89C102244424361
:10EFC80092FBF1F20AE7D3F8B82023E7D3F8CC2074
:10EFD800C3F8D42033E7002382F8A03047E7684617
:10EFE80020F007018D4601B50121064804F0DEF83E
:10EFF80018B10121034804F0E3F8BDE80140854653
:10F00800704700BF0004004007B500214FF4E070CE
:10F01800F9F779FF002140F2C110F9F774FF0021D8
:10F028004FF4E170F9F76FFF002140F2C310F9F7D0
:10F038006AFF002300931A4619461846F9F7CAFBD7
:10F0480003B05DF804FBB0F5804F3DBF034BD3F828
:10F05800DC3033F810004FF6FF707047EC260020C4
:10F06800834B002230B583F8A120824AC3F8DC2004
:10F0780010884FF6FF71884293B01D4605D047F6B9
:10F08800FE70125A8A4240F0E780FFF7BDFF002465
:10F0980004F1806000F5E030A1B24000013401F0D5
:10F0A800BBFCB4F5804FF3D101F0D4FB012385F804
:10F0B800D830FFF791FD704B01251D72F9F728F93B
:10F0C800002800F0CD80FFF731FD2946022002F02C
:10F0D80093FB6A48002403F096FB4FF4616304A98C
:10F0E80066480593ADF81040ADF81840ADF81240E9
:10F0F80003F012FC2A462946604804F072F82946B3
:10F108005E4803F0B2FC1D2303A88DF80C308DF87F
:10F118000D508DF80E508DF80F5002F0ADF82323E6
:10F1280003A88DF80C308DF80D408DF80E508DF831
:10F138000F5002F0A1F82946284602F045FB504B33
:10F148000893504B0793102309934FF480630E9351
:10F158004FF480730D9380230C9320230F9307A9FA
:10F168004FF44053484810931194ADF828500B942D
:10F1780001F0FEF92A460221444803F057FA2946CD
:10F18800414801F020FA0C230093C82204230A21E5
:10F198002046FAF756FD4FF00A1256212046FAF794
:10F1A800DAFC4FF4FA7258212046FAF7D4FC4FF4EF
:10F1B800041207212046FAF7CEFC354A08212046DA
:10F1C800FAF7C9FC4FF6FF7268212046FAF7C3FC2C
:10F1D8004FF4406221462046FAF7BDFC082120463C
:10F1E800FAF7D9FC224669212046FAF7B4FC4FF613
:10F1F800FF7268212046FAF7AEFC4FF46742692196
:10F208002046FAF7A8FC08212046FAF7C4FC6A2130
:10F218002046FAF7C0FC6B212046FAF7BCFC4FF4F5
:10F22800804254212046FAF796FC22465021204677
:10F23800FAF791FC174B4FF4C8625A6483F84040C0
:10F2480083F841400622019400944023632120461C
:10F25800FAF75EFC13B030BD012283F8D82028E706
:10F26800FFF764FC0C4B4FF48042DA61F2E700BF11
:10F27800EC2600200080030848000020000400401D
:10F28800942700200C380040580002400038004005
:10F298000D081010D02E0020902E002000B979E41F
:10F2A80000207047024BB3F8E20080B2704700BFFD
:10F2B800EC2600204FF480407047062921D8DFE86B
:10F2C80001F004080C1014181C000F4BD3F8E400CC
:10F2D80070470D4BD3F8E80070470B4BD3F8EC00A0
:10F2E8007047094BD3F8F0007047074BD3F8F40088
:10F2F8007047054BD3F8F8007047034BD3F8FC0070
:10F3080070470020704700BFEC26002000280ADD67
:10F31800054B1A68904206DC58601A685B68D31A75
:10F32800024AC2F89C30704748000020EC260020B2
:10F3380000280DDD074B5A68904209DB064A9042C7
:10F3480006DC18601A685B68D31A044AC2F89C3055
:10F35800704700BF4800002080841E00EC26002073
:10F36800FF2808B509D804F08BFB044B002204F0F1
:10F3780017FD04F0FDFD024B986108BD000009402F
:10F388004800002037B50C23009304460423C82204
:10F398000A210020FAF755FC424D14B30021084613
:10F3A8004FF48052FAF7D7FB3F4B5421DA6900201B
:10F3B800FAF7D1FB002210465021FAF7CCFB6A6C11
:10F3C800FF21082385F8401085F84130019100930A
:10F3D8006321D3B20020C2F30722FAF799FB03B0E6
:10F3E80030BD20464FF00A125621FAF7B4FB2046EA
:10F3F8004FF4C8625821FAF7AEFB20464FF40412C6
:10F408000721FAF7A8FB2046284A0821FAF7A3FBA8
:10F4180020464FF6FF726821FAF79DFB4FF44062D1
:10F4280021462046FAF797FB08212046FAF7B3FB56
:10F43800224620466921FAF78EFB20464FF6FF72D6
:10F448006821FAF788FB4FF4674220466921FAF7EA
:10F4580082FB08212046FAF79EFB6A212046FAF72C
:10F468009AFB6B212046FAF796FB6A6C85F84040B8
:10F47800072385F841308DE818002046D3B2632170
:10F48800C2F30722FAF744FB20464FF48042542186
:10F49800FAF761FB22465021204603B0BDE8304010
:10F4A800FAF759BBD02E0020902E00200D0810101E
:10F4B800F7B5D24C94F80031013B042B67D8DFE84C
:10F4C80013F0050068008E0096005401CC4B00250F
:10F4D8001D7284F8D850FAF7CFFCFAF7FFFB012029
:10F4E800FFF750FF2B462A46294601200095F9F7D9
:10F4F80071F980222B460192009206212846FAF7DC
:10F5080007FB012220212846FAF725FB4FF4FA20B1
:10F51800FAF7C2FC282102462846FAF71CFB2846BF
:10F52800FAF7B8FC242102462846FAF714FB012210
:10F5380020212846FAF70FFB2846FAF7ABFC2421CE
:10F5480002462846FAF707FB50212846FAF723FB1C
:10F55800212102462846FAF7FEFA2A46372128468C
:10F56800FAF7F9FA052220212846FAF7F4FA4FF4B7
:10F578004840FAF78FFC242102462846FAF7EBFAAE
:10F58800C4F804510223C4F8085184F8003103B0C8
:10F59800F0BD0F210020FAF7FEFAC007F7D5792150
:10F5A8000020FAF7F8FA7F2805DCC0F18000C4F8DB
:10F5B80004010323E9E7B0F5C07F02DAC0F5C070A3
:10F5C800F5E7B0F5207F02DAC0F52070EFE7B0F577
:10F5D800607FB4BFC0F56070C0F59060E7E7D4F80D
:10F5E800042137210020FAF7B6FA0423CDE70F21CA
:10F5F8000020FAF7D0FAC107C9D5D4F80831B3F515
:10F60800C87F28D221210020FAF7C5FA4FF44842D2
:10F61800D4F8081190FBF2F303FB1200104404EB3A
:10F62800810190FBF2F302FB1300A1F80E01D4F85C
:10F638000851FFF7AFFAD4F8043103F58073C4F822
:10F648000431D4F8083104EB85050133A5F80C0121
:10F65800C4F80831ADE76B4B997D9A7A01915B7AD2
:10F668000093002306211846FAF752FA00238CE784
:10F6780019461D8831F8046FAE4200F1010006D228
:10F68800D1F800E05E889D80C3F800E0DE800B467C
:10F698009042EDDB013A69D1B4F82A14B4F80E515E
:10F6A800B4F80C016FF000424FF00043A94284E81F
:10F6B8000C00B4F828245DD9C1F580432B4407EE2B
:10F6C800903AC2F58043B8EEE77A034407EE903AE1
:10F6D800F8EEE77A0132C7EE276A0E464FF0010EC0
:10F6E80043F6FF7CDFED487A9FED487A66EEA77A0D
:10F6F800F4EEC77AF1EE10FA44BFBDEEE77A17EEE2
:10F70800103A9FED437A48BF2360F4EEC77AF1EED2
:10F7180010FAC4BFFDEEE77AC4ED017A824234D113
:10F7280072B6FFF771FC2946B4F80E31B4F80C2113
:10F73800384D0020FFF794F9FB88BA88798837F8A4
:10F74800040BFFF78DF9BD42F6D133464FF48042E2
:10F75800B4F82A14B4F82804FFF782F962B601F065
:10F7680079F8012384F8D83080E7C7222A4F00208F
:10F778003B468DE7C5F580430B4407EE903AC0F54C
:10F788008043B8EEE77A1344A0E7EAB907EE90EAB7
:10F79800B8EEE77A07EE901AF8EE677AE6EE877A1F
:10F7A800FDEEE77A17EE905A6B42C3F30D03C5F3EB
:10F7B8000D0558BF5D42ADB20132B2F5804F0EF172
:10F7C800010EA8BF0022A9E76245F5D107EE90EA2D
:10F7D800B8EEE77A07EE901AF8EE677AE6EE877ADF
:10F7E800FDEEE77A17EE903A5E4206EA020603EA71
:10F7F800020358BF73429EB2DEE700BFEC2600202A
:10F8080048000020902E002000007A440000004F9D
:10F81800000000CF142B0020F8270020024B012203
:10F8280083F80021704700BFEC260020044B93F8B2
:10F83800002102F0FF0012B1D3F80801013070472F
:10F84800EC260020014B1868704700BFEC2600200A
:10F85800014B5868704700BFEC26002048B9064B9A
:10F868001B7A1BB1054BD3F8C80070476621FAF71D
:10F8780092B90020704700BF48000020EC26002005
:10F88800B0F5C87F3FBF064B03EB8000B0F80C31E2
:10F89800B0F80E0134BF40EA03404FF0FF30704724
:10F8A800EC260020014B1872704700BF480000206A
:10F8B800014B83F8D8007047EC26002000000000B8
:10F8C80030B501219BB0022001F07EFF01214FF0ED
:10F8D800805001F079FF01214FF0005001F074FFD2
:10F8E8004FF4887001F0FCFE434801F0F9FE002453
:10F8F80003236946414800938DF804308DF807408A
:10F9080001F07EFA3E4B10933E4B0F934FF4806309
:10F9180016934FF4807315930223ADF84830802373
:10F9280014930FA92023384817931194199413940A
:10F93800189400F01DFE0121334800F044FE012117
:10F94800324800F0F4FAF8F7B5FC0446F8F7B2FCD0
:10F95800001B0028B8BF40420428F7DD2B480021CF
:10F9680000F0D1FA294800F0C3FA284800F0D3FA89
:10F9780004460028F9D1022502A9029003900490B8
:10F988008DF818002148059500F074FA07A800F0D2
:10F9980047FA4FF4005307A91C48079308940994A1
:10F9A8000A940B940C940D948DF8385000F01AFAC0
:10F9B8002946164800F0A9FC0121144800F09CFCD7
:10F9C800032301220C21114800F088FB01210F4874
:10F9D80003232A4600F082FB01210C4800F07FFA3D
:10F9E80001210A4800F007FD0028F9D0074800F077
:10F9F800E3FB1BB030BD00BF00220010000400482C
:10FA0800382E0020400400505804024000040050E2
:10FA1800082808B503D009280CD0002008BD1E4BC3
:10FA2800188883B240F26B10584340F6FF7390FB7E
:10FA3800F3F008BD184B588880B207EE900AF8EE2C
:10FA4800677A17EE900A04F02DF80DA3D3E9002386
:10FA580004F07CF80CA3D3E9002304F0A1F904F026
:10FA6800AFFA04F01FF800220C4B03F0BBFE08A30A
:10FA7800D3E9002304F094F904F07AFA08BD00BF32
:10FA88006666666666660A400000000000FEAF40D3
:10FA98007B14AE47E17A843F382E00200000E03F17
:10FAA800F0B510208BB001F02BFE224D01214FF450
:10FAB800001001F0A1FE01214FF4802001F084FE26
:10FAC80028460422062101F013FA042228460721B9
:10FAD80001F00EFA02230AAE8DF8083003238DF8E0
:10FAE8000930402346F8243D0024012731462846A2
:10FAF8008DF80A708DF80B4001F082F928460E4DFA
:10FB080080233146019301F07BF9284601F002FA7F
:10FB18000AA90A4B41F81C3D28460694049405940A
:10FB28000894099401F012FA3946284601F049FA76
:10FB38000BB0F0BD00040048005400407A25E000F6
:10FB48002DE9F74305460C4616461F464FF400417B
:10FB5800284601F068FB80460028F7D15FFA86F94D
:10FB68004FF41053BFB200934A464FF00073394622
:10FB7800284601F0DAFA2644B44203D1012003B042
:10FB8800BDE8F0830421284601F04DFB0028F9D098
:10FB9800284601F03BFBCDF8008004F8010B4FF03C
:10FBA80000734A463946284601F0BFFAE4E72DE9D2
:10FBB800F74305460C4616461F464FF400412846B3
:10FBC80001F031FB80460028F7D15FFA86F94FF43F
:10FBD8000053BFB200934A464FF000733946284697
:10FBE80001F0A3FA2644B44203D1012003B0BDE8D2
:10FBF800F0830221284601F016FB0028F9D014F8FA
:10FC0800011B284601F000FBCDF800804FF000737F
:10FC18004A463946284601F088FAE4E77047FEE785
:10FC2800FEE7FEE7FEE7704770477047384AD2F8AC
:10FC3800883043F47003C2F88830364B1A6842F0B3
:10FC480001021A605968344A0A405A601A6822F058
:10FC5800847222F480321A601A6822F480221A60B0
:10FC68005A6822F4FE025A60DA6A22F00F02DA6257
:10FC7800196B2A4A82B00A401A6300229A600092DD
:10FC880001921A6842F480321A601A6802F400324B
:10FC98000192009A01320092019A1AB9009AB2F5BB
:10FCA800A06FF2D11A6812F4003218BF0122019233
:10FCB800019A012A04D0164B194A9A6002B070477B
:10FCC800184A122111605A685A605A685A605A686C
:10FCD80042F480625A605A6822F47C125A605A6868
:10FCE80042F4F8125A601A6842F080721A601A6870
:10FCF8009201FCD55A6822F003025A605A6842F011
:10FD080002025A605A6802F00C02082AFAD1D2E7B5
:10FD180000ED00E0001002400CC07FF8CCFC00FFB2
:10FD280000800008002002401549164A4B6803F07D
:10FD38000C03042B10B50CD0082B0CD0124B1360FD
:10FD48004B68C3F30313134419791368CB4013604A
:10FD580010BD0E4BF3E74B684868C00349BFC86A3B
:10FD68000B480A4C00F00F00C3F3834348BF01302F
:10FD780003F1020348BFB4FBF0F04343DFE700BFE1
:10FD8800001002406400002000127A000024F400F1
:10FD980000093D00B0F1A04F08B502D00F4B9842C2
:10FDA8000BD101214FF0805001F032FD00214FF0BE
:10FDB8008050BDE8084001F02BBD094B984203D0A4
:10FDC80003F58073984208D101214FF0005001F0EB
:10FDD8001FFD00214FF00050EBE708BD0001005067
:10FDE80000040050C3680D4A10B51A4091E8180085
:10FDF80023438C682343CC6823430C6923434C6911
:10FE080023438C6923431343C360026B0B7F22F0A7
:10FE18000F02013B1343036310BD00BF07C0FFFD82
:10FE28000023036043608360C360036143618361AF
:10FE3800012303777047C36C91E80C001343CA6829
:10FE480043EA02230A6943EA82334A6943EA0253CE
:10FE58008A6943EA82630A7A013A1343C3647047A2
:10FE680000230360436001230372C360036143619D
:10FE780083617047B0F1A04F10B5114B02D0114A01
:10FE8800904218D1104A94681C4091E80C00134322
:10FE98008A681343CA6843EA02330A7CB0F1A04F68
:10FEA80043EA022343EA040302D0064A904204D1FB
:10FEB800054A936010BD054AE5E7044AF9E700BF23
:10FEC800E010FCFF00010050000300500007005044
:10FED8000023036043608360C360037470478368D2
:10FEE80019B143F001038360704743F00203FAE756
:10FEF800836843F0004383607047D0F8B4007047CC
:10FF0800C0F8B4107047836823F080438360836827
:10FF18001943816070478068C00F7047836843F059
:10FF28000203836070478068C0F3400070478368AD
:10FF380023F040538360836819B143F08053836092
:10FF4800704743F00053FAE7012332B1D0F8B020EC
:10FF58008B401343C0F8B0307047D0F8B0208B40C6
:10FF680022EA0303F6E7C36819B143F40013C36038
:10FF7800704723F40013FAE7C36819B143F48043C8
:10FF8800C360704723F48043FAE7C36823F0E07343
:10FF98001943C1607047036A23F07F6323F4702319
:10FFA8000362036A43EA01410162036A23F47F633F
:10FFB80023F00F030362036A1A4302627047436A1D
:10FFC80023F47F034362436A43EA01414162436A7F
:10FFD80023F0FF034362436A1A4342627047836A0D
:10FFE80023F47F038362836A43EA01418162836A5F
:08FFF80023F0FF038362836A1A
:020000040801F1
:100000001A4382627047C36823F0F84343EA816170
:10001000C160704710B5D0F8A020D0F8A0400123EF
:1000200003FA01F1A3F50023214313401943C0F85B
:10003000A01010BD10B5D0F8A420D0F8A440012322
:1000400003FA01F1A3F50023214313401943C0F83B
:10005000A41010BDB0F1A04F02D0074B984206D1BA
:10006000064B9A6829B142F400029A607047044B2B
:10007000F7E722F40002F8E7000100500003005007
:1000800000070050B0F1A04F02D0074B984206D1B4
:10009000064B9A6829B142F480029A607047044B7B
:1000A000F7E722F48002F8E7000100500003005057
:1000B00000070050B0F1A04F02D0074B984206D184
:1000C000064B9A6829B142F080729A607047044BDF
:1000D000F7E722F08072F8E70001005000030050BB
:1000E00000070050042A30B51CD802EB4202046B12
:1000F00052001F25954024EA050401FA02F222432A
:100100000263092939D90A398269826901EB4101FF
:1001100007248C4022EA0402826182698B401343E7
:10012000836130BD092A0CD80624053A6243456B29
:100130001F24944025EA040401FA02F22243426398
:10014000DFE70E2A4FF006040BD80A3A6243856BAC
:100150001F24944025EA040401FA02F22243826338
:10016000CFE70F3A6243C56B1F24944025EA04048D
:1001700001FA02F22243C263C3E7013942694269CC
:1001800001EB410138248C4022EA040242614269B9
:10019000033103FA01F11143416130BD036B23F0D8
:1001A0000F030363036B0139194301637047C3688D
:1001B00023F47C63C360C3680A431A43C260704778
:1001C000836843F00403836070478068C0F3800055
:1001D0007047836843F0100383607047C368013938
:1001E00023F4602343EA4143C3607047C36819B1F5
:1001F00043F48033C360704723F48033FAE7006C24
:1002000080B27047B0F1A04F02D0044B984202D1A7
:10021000034BD8687047034BFBE700BF0001005059
:100220000003005000070050036E23F0F8430366FC
:10023000036E43EA81610166036E23F47F6323F05A
:100240000F030366036E1A4302667047436E23F082
:10025000F8434366436E43EA81614166436E23F48B
:100260007F6323F00F034366436E1A434266704771
:10027000836E23F0F8438366836E43EA816181666F
:10028000836E23F47F6323F00F038366836E1A4328
:1002900082667047C36E23F0F843C366C36E43EAB9
:1002A0008161C166C36E23F47F6323F00F03C366CD
:1002B000C36E1A43C2667047036E19B143F0004320
:1002C0000366704723F00043FAE7436E19B143F029
:1002D00000434366704723F00043FAE7836E19B189
:1002E00043F000438366704723F00043FAE7C36E90
:1002F00019B143F00043C366704723F00043FAE7A7
:10030000C36819B143F00103C360704723F00103D0
:10031000FAE7C36823F00203C360C3681943C160EE
:100320007047092970B519D9A1F10A04856904EB50
:1003300044040726A64025EA060503FA04F42C43E4
:100340008461541E06226243C36C4FF4F8549440F7
:1003500023EA040391401943C16470BD456901EB70
:1003600041060724B44025EA040503FA06F42C43A9
:100370004461E6E7C36C013923F003031943C16408
:100380007047C36C23F0FC03C364C36C0A431A4375
:10039000C2647047836843F00803836070478368D2
:1003A00043F02003836070478068C0F3C00070474B
:1003B000C36819B143F00073C360704723F0007342
:1003C000FAE7C36819B143F48013C360704723F49C
:1003D0008013FAE782B0002301930190019B8033E0
:1003E00019440191019B186880B202B070474368BC
:1003F00012B119434160704723EA0101FAE703682B
:100400000B4214BF01200020704701607047B0F11B
:10041000A04F02D0054B984206D1054B1B680B42FA
:1004200014BF012000207047024BF7E70001005085
:100430000003005000070050B0F1A04F02D0064B5F
:10044000984204D1054B1A68114319607047044A59
:1004500013681943116070470001005000030050F9
:10046000000700500368426889B211EA030003D014
:10047000114214BF01200020704703681943016036
:10048000704700BF036823F001031B041B0C0360CB
:100490000023036043608360C360294B984204D10A
:1004A000284A536843F00F0326E0274B984204D1B3
:1004B000244A536843F0F0031EE0244B984204D1D1
:1004C000204A536843F4706316E0214B984204D1EC
:1004D0001C4A536843F470430EE01E4B984204D10B
:1004E000184A536843F4702306E01B4B984205D129
:1004F000144A536843F4700353607047174B984293
:1005000004D1104A536843F07063F5E7144B9842E6
:1005100001D1144AC5E7144B984201D1114AC8E7EA
:10052000124B984201D10F4ACBE7114B984201D1AF
:100530000C4ACEE70F4B9842DFD10A4AD1E700BF01
:1005400008000240000002401C000240300002404F
:1005500044000240580002406C000240800002400B
:1005600008040240000402401C040240300402401F
:1005700044040240580402408B68026810B50C6ABB
:1005800023430C6923434C6923438C692343CC697F
:1005900023434C6A23438C6A22F4FF4222F0700208
:1005A0002343134303608B8943600B6883604B686C
:1005B000C36010BD002303604360836083810361D7
:1005C00043618361C361036243628362704703686E
:1005D00019B143F001030360704723F001031B04CA
:1005E0001B0CF8E741607047406880B270470368B1
:1005F00012B119430160704723EA0101FAE7C30011
:100600004CBF044B044B1B68034214BF0120002065
:10061000704700BF0004024000000240FFF7EFBF38
:10062000C3004CBF014B024B5860704700040240AE
:1006300000000240FFF7F4BF0A4B4FF0FC521A6073
:100640006FF0FC5100225A609A60DA601A615961B9
:100650000C2119625A629A62DA621A6303225A639F
:10066000704700BF000401408279036870B50479C7
:10067000002A64D023F01F0101F1804101F582318D
:1006800003F01F020D68012303FA02F225EA0202B9
:100690000A600168324D21F01F0601F01F017259F6
:1006A00003FA01F122EA01017151016804F180426B
:1006B00021F01F0502F5823201F01F01AC5803FA48
:1006C00001F12143A9500268264D22F01F0402F0D7
:1006D0001F02615903FA02F221EA02026251026822
:1006E000214C22F01F0602F01F02315903FA02F2D8
:1006F00021EA0202417932511029026812D122F016
:100700001F0102F01F024E5903FA02F232434A510E
:10071000026822F01F0102F01F02085993400343B0
:100720000B5170BD01F1804122F01F0001F58231B3
:1007300002F01F02445893402343435070BD04F11C
:10074000804223F01F0502F5823203F01F03A958EF
:10075000012000FA03F321EA0303AB5070BD00BF90
:1007600004040140080401400C040140002310224D
:100770000360037142718371704720F01F0110B54F
:10078000044A00F01F038C580120984020438850F1
:1007900010BD00BF1004014020F01F02054B00F007
:1007A0001F00D258012303FA00F0104214BF18466C
:1007B000002070471404014020F01F0303F1804320
:1007C00003F5823300F01F00012282401968586946
:1007D000104003D0114214BF01200020704720F0C8
:1007E0001F02012300F01F0003FA00F0014BD0505C
:1007F000704700BF14040140FFF7F1BF034A1368BC
:1008000023F0030318431060704700BF002002402C
:10081000044B1A6818B142F008021A60704722F0BF
:100820000802FAE700200240044B1A6818B142F0AF
:1008300010021A60704722F01002FAE7002002400E
:10084000044B1A69120641BF034A5A6002F188320A
:100850005A6070470020024023016745024A13692D
:1008600043F080031361704700200240044B1A6973
:1008700092055FBF034A9A6002F188329A6070471E
:100880000020024023016745024A136923F40073E4
:100890001361704700200240024A136943F4005379
:1008A0001361704700200240024BD869C0F3072053
:1008B000704700BF00200240014B186A704700BF1C
:1008C00000200240034BDB6913F0060F14BF012028
:1008D0000020704700200240044B1A6911B11043F8
:1008E0001861704722EA0000FAE700BF00200240CA
:1008F000034BDB68034214BF01200020704700BF98
:1009000000200240014BD860704700BF0020024029
:10091000084BDA68D10709D4DA68D20608D4DB6854
:1009200013F0040F14BF0320042070470120704708
:10093000022070470020024010B50446FFF7E8FF90
:10094000012806D10CB9052010BDFFF7E1FF013CDD
:10095000F6E7002C08BF052010BD38B505464FF45A
:100960003020FFF7E9FF042811D1094C236943F037
:10097000020323616561236943F0400323614FF45F
:100980003020FFF7D9FF236923F00203236138BD2C
:100990000020024010B54FF43020FFF7CDFF0428AF
:1009A00010D1094C236943F004032361236943F008
:1009B000400323614FF43020FFF7BEFF236923F08B
:1009C0000403236110BD00BF0020024073B5002363
:1009D00006464FF430200D460193FFF7ADFF042883
:1009E00019D10E4C236943F001032361ABB233806C
:1009F0004FF43020FFF7A0FF042808D102360196FB
:100A0000019B2D0C1D804FF43020FFF795FF2369CB
:100A100023F00103236102B070BD00BF002002403B
:100A200070B505464FF430200E46FFF785FF0428C9
:100A30000DD1074C236943F0010323614FF43020AB
:100A40002E80FFF779FF236923F00103236170BD36
:100A50000020024038B5FFF735FF00284FF4302062
:100A60000CBFAA250025FFF767FF042822D1124CEE
:100A7000236943F020032361236943F0400323618A
:100A80004FF43020FFF758FF04280DD1236923F0DD
:100A900020032361236943F010032361074B4FF4C4
:100AA00030201D80FFF748FF05281EBF236923F073
:100AB0001003236138BD00BF0020024000F8FF1F73
:100AC00010B504464FF43020FFF736FF04281DD13F
:100AD0001249E4430B69E2B243F01003FF2A0B61B1
:100AE0000AD1C4F30724FF2C11D104200B4A136947
:100AF00023F01003136109E0094B4FF430201A81F1
:100B0000FFF71AFF0428ECD00528EFD110BD044BE5
:100B10004FF430205C81FFF70FFFF5E70020024023
:100B200000F8FF1F38B505464FF43020FFF704FFEB
:100B3000042823D1154C236943F020032361236942
:100B400043F0400323614FF43020FFF7F5FE042803
:100B500015D1236923F020032361236943F0100397
:100B600023610B4BADB21D804FF43020FFF7E4FE44
:100B7000052803D0236923F01003236138BD05281D
:100B8000FCD0236923F02003F7E700BF00200240D8
:100B900000F8FF1FF8B5124C124BA36003F1883325
:100BA0000546A3604FF430200E461746FFF7C4FEFB
:100BB000042814D1236967F0070743F010033E436C
:100BC00023613543084BEDB25D804FF43020FFF7D1
:100BD000B3FE05281EBF236923F010032361F8BD6F
:100BE000002002402301674500F8FF1F38B5104C74
:100BF000104BA36003F188330546A3604FF4302007
:100C0000FFF79AFE042811D1236943F010032361F2
:100C1000094B45F0EF055D804FF43020FFF78CFE67
:100C200005281EBF236923F01003236138BD00BFD0
:100C3000002002402301674500F8FF1F38B5104C23
:100C4000104BA36003F188330546A3604FF43020B6
:100C5000FFF772FE042811D1236943F010032361CA
:100C6000094B45F0DF055D804FF43020FFF764FE4F
:100C700005281EBF236923F01003236138BD00BF80
:100C8000002002402301674500F8FF1F38B50546E4
:100C90004FF43020FFF750FE042812D1094C23698D
:100CA00043F010032361084B45F0BF055D804FF40E
:100CB0003020FFF741FE05281EBF236923F01003F3
:100CC000236138BD0020024000F8FF1F38B5104CEA
:100CD000104BA36003F188330546A3604FF4302026
:100CE000FFF72AFE042811D1236943F01003236182
:100CF000094B45F088055D804FF43020FFF71CFE5E
:100D000005281EBF236923F01003236138BD00BFEF
:100D1000002002402301674500F8FF1F70B506461A
:100D20004FF430200D46FFF707FE042810D1094C80
:100D30002369ADB243F0100323614FF430203580B6
:100D4000FFF7FAFD05281EBF236923F01003236176
:100D500070BD00BF00200240B0F1904F08B50BD12C
:100D600001214FF4003000F057FD00214FF4003016
:100D7000BDE8084000F050BD1E4B984208D101214B
:100D80004FF4802000F048FD00214FF48020EFE771
:100D9000194B984208D101214FF4002000F03CFD8E
:100DA00000214FF40020E3E7144B984208D10121C1
:100DB0004FF4801000F030FD00214FF48010D7E791
:100DC0000F4B984208D101214FF4001000F024FD90
:100DD00000214FF40010CBE70A4B984208D10121C3
:100DE0004FF4800000F018FD00214FF48000BFE7B1
:100DF00008BD00BF0004004800080048000C00487F
:100E000000100048001400482DE9F04100230F684D
:100E10001D464FF0010E03260EFA05FC3CEA0702C0
:100E200034D10C79621E012A19D8826806FA03F8B7
:100E300022EA080282604A79D0F808809A4042EAA1
:100E400008028260828892B222EA0C0282808A7949
:100E5000B0F804C0AA4042EA0C0292B28280D0F8F4
:100E600000C006FA03F2D24302EA0C0CC0F800C03C
:100E7000D0F800C09C4044EA0C040460C4682240DE
:100E8000C260CA79C4689A402243C2600135102DFD
:100E900003F10203C0D1BDE8F0814FF6FF73036098
:100EA00001220023037142718371C371704741F4C1
:100EB0008033C361C161C361C369C3697047038A79
:100EC000194214BF012000207047008A80B2704789
:100ED000838A194214BF012000207047808A80B2A3
:100EE000704781617047018570470AB18161704721
:100EF000018570478182704701F00703C90800EB44
:100F0000810010B5016A9B000F249C4021EA040176
:100F10000162016A9A400A43026210BD08B50C4B97
:100F200098424FF001010AD14FF4001000F08CFC00
:100F300000214FF40010BDE8084000F085BC4FF4DC
:100F4000800000F081FC00214FF48000F3E700BF37
:100F5000005400400368164A23F00103036003684D
:100F600010B51A408C684B6843EA042313430360AE
:100F70000B680A6923F070630361036843F001039F
:100F8000036000238360C3608B69134383608368BD
:100F9000CA6843F4004383600368134303604368F3
:100FA0004A6923F0784323F400431343436010BDA0
:100FB000FFE0CF0000234FF40042036043608360F2
:100FC000C3600361426183617047036819B143F0F4
:100FD00001030360704723F00103FAE7036823F07D
:100FE000010303600368036843F001030360704773
:100FF000036819B123F400330360704743F40033EE
:10100000FAE7036819B143F480230360704723F4BF
:101010008023FAE7C36819B143F40043C360704703
:1010200023F40043FAE7C368120223F4FF6302F4D7
:10103000E06201F0FE0123F006030A431A43C26096
:101040007047036819B143F400230360704723F429
:101050000023FAE7036819B143F480330360704753
:1010600023F48033FAE7436823F47F7323F0030308
:10107000C1F309010B4343607047436819B143F45E
:1010800000634360704723F40063FAE7436819B1D3
:1010900043F000734360704723F00073FAE743683E
:1010A00019B143F080734360704723F08073FAE70F
:1010B000436823F47F0343EA01414160704743687A
:1010C00019B923F480634360704743F48063FAE7FF
:1010D000436819B143F400534360704723F400534D
:1010E000FAE7436819B143F480434360704723F43F
:1010F0008043FAE7436819B143F480534360704773
:1011000023F48053FAE7436819B123F400434360A2
:10111000704743F40043FAE78069000C00F0FE00DA
:101120007047836913F4803F14BF4FF48060002040
:10113000704730B54468039D24F07F7424F459341B
:10114000C1F309012B4324F47F74194324F00304F1
:1011500041EA02412143416030BD036819B143F4C3
:1011600080030360704723F48003FAE7436919B1F1
:1011700043F400434361704723F40043FAE74369B3
:1011800019B143F000434361704723F00043FAE78D
:10119000436919B143F480534361704723F480538A
:1011A000FAE7436923F47F6323F00F03C1F30B01D4
:1011B0000B43436170474269044B22F07F6222F483
:1011C000702203EA01411143416170470000FF0FA3
:1011D000036819B143F400030360704723F400036C
:1011E000FAE7036819B143F080630360704723F0A6
:1011F0008063FAE7006AC0B2704782B000230193AF
:101200000190019B19440191019B186802B070473D
:1012100081627047406AC0B27047036812B11943D7
:101220000160704723EA0101FAE7FFF7F6BF83691F
:101230000B4214BF012000207047C161704711F4B8
:101240007C5F036808D003F080038069084002D007
:10125000181C18BF0120704711F0C00F14BF03F015
:1012600040030B40F1E7C161704700BF40F0BF6031
:10127000024B40F40030D860704700BF00ED00E042
:1012800010B5C2780378E2B1124AD168427880780A
:10129000C943C1F30221C1F10404A2400F2424FA7E
:1012A00001F101400A430C491201C818D2B280F87A
:1012B000002303F01F005A090123834041F8223024
:1012C00010BD5A09012103F01F0301FA03F3203274
:1012D0000149F3E700ED00E000E100E021F06041AA
:1012E00021F07F01014B01439960704700ED00E060
:1012F000044B1A6911B110431861704722EA0000CB
:10130000FAE700BF00ED00E0044B1A6804280CBFA8
:1013100042F0040222F004021A60704710E000E07C
:10132000114B1A6842F001021A6059680F4A0A40CC
:101330005A601A6822F0847222F480321A601A68A5
:1013400022F480221A605A6822F4FE025A60DA6A95
:1013500022F47F5222F03F02DA62196B044A0A40FB
:101360001A6300229A6070470010024000C0FFF824
:10137000CCFC000F024B00221A701870704700BF9F
:1013800002100240034A136823F0F80343EAC00046
:101390001060704700100240014B1860704700BF9A
:1013A00000004242064B1A6A22F001021A621A6ACF
:1013B00022F004021A621A6A10431862704700BFD2
:1013C00000100240044B1A6A22F018021A621A6ACC
:1013D00010431862704700BF00100240014B1860B4
:1013E000704700BF80044242044A536823F47413D8
:1013F0005360536819430143516070470010024025
:10140000014B1860704700BF60004242034AD36A34
:1014100023F00F031843D062704700BF0010024052
:10142000014B1860704700BF4C004242014B1870DE
:10143000704700BF07100240034A536823F00303BC
:1014400018435060704700BF00100240024B5868BC
:1014500000F00C00704700BF00100240034A5368C0
:1014600023F0F00318435060704700BF00100240A3
:10147000034A536823F4E06318435060704700BF89
:1014800000100240034A536823F4605343EAC0004B
:1014900050607047001002408E4B5A6802F00C02F8
:1014A000042AF0B578D0082A7AD08B490160002A46
:1014B00074D15968894CC1F3031114F801E0016833
:1014C0005FFA8EFE21FA0EF545605E68C6F30226CD
:1014D000A65D25FA06F686605F68C7F3C227E75D5A
:1014E000FFB2FD40C560D3F82CC0CCF3041C04EB64
:1014F0004C0CBCF810C01FFA8CFC1CF0100F0EBF77
:101500000161B2FBFCFCC0F810C0D3F82CC0CCF3D6
:10151000442C04EB4C04248AA4B214F0100F0EBF28
:101520004161B2FBF4F444611C6BE4065ABF6A4C9F
:10153000846181611C6BA4065ABF674CC461C161A0
:101540001C6BE40541D58A423FD1BE453DD15400D4
:1015500004621C6BA4053AD58A4238D1BE4536D107
:101560004A0042621A6B920733D185621A6B12F4F9
:10157000403F45D1C6621A6B12F4402F5AD1066320
:101580001A6B12F4401F6FD146631A6B12F4400FAE
:1015900040F085808663F0BD514A0260002288E7F2
:1015A0005A685968C90349BFD96A4E494C4C01F081
:1015B0000F01C2F3834248BF013102F1020248BF6A
:1015C000B4FBF1F14A43026073E70562C1E745628B
:1015D000C8E71A6B02F00302012A01D18162C5E754
:1015E0001A6B02F00302022A03D14FF40042826216
:1015F000BCE71A6B02F00302032AB7D1364AF6E7BA
:101600001A6B02F44032B2F5803F01D1C162B2E7F9
:101610001A6B02F44032B2F5003F03D14FF400429E
:10162000C262A8E71A6B02F44032B2F5403FA2D181
:10163000294AF5E71A6B02F44022B2F5802F01D156
:1016400001639DE71A6B02F44022B2F5002F03D12B
:101650004FF40042026393E71A6B02F44022B2F5A2
:10166000402F8DD11C4AF5E71A6B02F44012B2F5F7
:10167000801F01D1416388E71A6B02F44012B2F572
:10168000001F03D14FF4004242637EE71A6B02F45D
:101690004012B2F5401F7FF478AF0F4AF4E71A6B9F
:1016A00002F44002B2F5800F01D18163F0BD1A6BE4
:1016B00002F44002B2F5000F03D14FF400438363FC
:1016C000F0BD1B6B03F44003B3F5400FF8D1024BA0
:1016D000F5E700BF0010024000127A0078000020F9
:1016E0000024F40000093D00030F064BDA6A14BF22
:1016F00022F4785222F4F872DA62DA6A1043D8627D
:10170000704700BF00100240030F064B1A6B14BF56
:1017100022F0200222F010021A631A6B10431863A1
:10172000704700BF00100240030F064B1A6B14BF36
:1017300022F4007222F480721A631A6B1043186349
:10174000704700BF00100240020F013A0F4B042AFD
:1017500008D8DFE802F0030B0F1317001A6B22F012
:1017600003021A631A6B1043186370471A6B22F452
:101770004032F6E71A6B22F44022F2E71A6B22F4A9
:101780004012EEE71A6B22F44002EAE70010024032
:10179000014B1860704700BFD8004242024A136AEA
:1017A00018431062704700BF00100240014B1860E0
:1017B000704700BFDC004242014B1860704700BF19
:1017C0003C044242014B1860704700BF4004424253
:1017D000044B5A6911B110435861704722EA000066
:1017E000FAE700BF00100240044B9A6911B11043A0
:1017F0009861704722EA0000FAE700BF001002403B
:10180000044BDA6911B11043D861704722EA000035
:10181000FAE700BF00100240044B9A6A11B110436E
:101820009862704722EA0000FAE700BF0010024009
:10183000044BDA6811B11043D860704722EA000007
:10184000FAE700BF00100240044B1A6911B11043BF
:101850001861704722EA0000FAE700BF001002405A
:10186000044B1A7811B110431870704722EA000037
:10187000FAE700BF091002404209094B07D11B6873
:1018800000F01F0023FA00F000F001007047012A69
:1018900001D11B6AF4E7042A0CBF5B685B6AEFE7BF
:1018A0000010024007B5002301931120FFF7E4FF69
:1018B000019B01330193019BB3F5A06F01D0002878
:1018C000F3D01120FFF7D8FF003018BF012003B07C
:1018D0005DF804FB024A536A43F080735362704719
:1018E00000100240034B9B68184214BF01200020E7
:1018F000704700BF00100240014B1870704700BFD6
:101900000A10024000230928DAB203F1010303D8C8
:1019100040EA0210C0B270470A38C0B2F3E70309C8
:1019200003EB830300F00F0000EB4300C0B27047ED
:1019300000217F22FF2380E80E007047044B10B186
:10194000FF225A627047CA225A625322F9E700BF47
:101950000028004082B0002301930D4BDA68520644
:1019600014D44FF0FF32DA601846DA680199013179
:1019700001910199B1F5005F02F0400201D0002A07
:10198000F3D0C068C0F3801002B070470120FBE7BD
:1019900000280040024AD36823F08003D3607047D8
:1019A0000028004038B50F4CCA236362532363629A
:1019B0000546FFF7CFFF88B1A36823F04003A3607B
:1019C000A3682A681343A360AB68236123696A682C
:1019D00043EA02432361FFF7DDFF0120014BFF22B1
:1019E0005A6238BD0028004013B500230193114B03
:1019F0009A6892061BD4CA225A6253225A62DA6843
:101A000022F0A002DA601C46DA68019901310191E6
:101A10000199B1F5004F02F0200201D0002AF3D065
:101A2000E068FF23C0F34010636202B010BD0120E4
:101A3000FBE700BF0028004037B51F4CCA23002534
:101A40000195636253236362FFF784FF28B9002086
:101A5000194BFF225A6203B030BD42F201132560D8
:101A60006360A36803F00703A3602346E26801995B
:101A7000013101910199B1F5005F02F0040201D03A
:101A8000002AF3D0DA685207E1D59A684FF6FF7161
:101A900000229A60596109491961DA611A62DA62B1
:101AA000DA635A649A64DA601A64FFF79DFF0030C3
:101AB00018BF0120CCE700BF00280040FF007F00D6
:101AC00038B50B4CCA236362532363620546FFF7A4
:101AD00041FF38B1A36845B143F01003A360FFF79D
:101AE00059FF0120FF23636238BD23F01003F5E79F
:101AF00000280040074BCA225A6253225A629A6851
:101B000028B142F020029A60FF225A62704702F028
:101B1000DF02F8E700280040224B0A789B6870B586
:101B20004D788C78B0B913F0400300D1CB701046DB
:101B3000FFF7E8FE06462846FFF7E4FE0546204686
:101B4000FFF7E0FECB7840EA034040EA064040EA77
:101B500005240AE013F0400300D1CB70280240EACC
:101B600002402043CC7840EA04440E4DCA236B6205
:101B700053236B62FFF7EEFE70B104F07F3424F064
:101B8000FE442C60FFF706FFAB689B0608D4FFF706
:101B90002BFF003018BF0120024BFF225A6270BD9C
:101BA0000120F9E7002800400023C3700370437050
:101BB00083707047104B70B51C6804F07F3323F0BE
:101BC000FE431D0C05F03F06C3F3062204F07F041C
:101BD00005F040050E704A708C70CD7058B93046D3
:101BE000FFF79DFE08701046FFF799FE48702046EB
:101BF000FFF795FE887070BD00280040014B986A81
:101C00005B6870470028004070B54B78CA788D78C3
:101C10000C78002833D1D80603D523F010030A33FB
:101C20004B701046FFF76EFE06464878FFF76AFED7
:101C300001462846FFF766FE40EA443040EA064087
:101C400040EA0124114DCA236B6253236B62FFF7F4
:101C500081FE70B124F07F4424F0C0046C60FFF773
:101C600099FEAB689B0608D4FFF7BEFE003018BF94
:101C70000120064BFF225A6270BD0120F9E71802CD
:101C800040EA0240284340EA4434DBE700280040B1
:101C900001230370837043700023C370704738B50D
:101CA0000F4B5A6822F07F4323F0C0031D0CC3F38F
:101CB000042402F03F02C3F34233CD704C708A70AB
:101CC0000B7058B92846FFF72AFEC8702046FFF768
:101CD00026FE48701046FFF722FE887038BD00BF10
:101CE000002800402DE9F047264B9468D2F804A064
:101CF000977892F800E092F80180167B154600BBB9
:101D00009B6813F0400300D1D3707046FFF7FAFDD3
:101D100081464046FFF7F6FD80463846FFF7F2FD64
:101D200007463046FFF7EEFDEB7844EA0A0444EA42
:101D300003433B4343EA094343EA082343EA006081
:101D400010E09A6812F0400200D1EA7044EA0A00FA
:101D5000384340EA0E40EB7840EA082040EA03406E
:101D600040EA0660074BCA225A6253225A62B1F512
:101D7000807F4FF0FF020CBFD86118625A62BDE845
:101D8000F08700BF0028004000230122C3700370C9
:101D9000437083708360027343607047F8B5174BDC
:101DA000B1F5807F0CBFDB691B6AC3F307410646B0
:101DB00001F03F0001F04001C3F3062503F07F046A
:101DC00003F08047D170C3F3056103F080331070D6
:101DD0005570947011739760536076B9FFF79FFD4B
:101DE00010702846FFF79BFD50702046FFF797FDC7
:101DF00090700846FFF793FD1073F8BD002800406F
:101E000013B500230193134BCA225A6253225A621C
:101E10009A6839B11043986001200E4BFF225A6234
:101E200002B010BD22EA00029A60000A1C46DA687D
:101E30000199013101910199B1F5005F02EA0002B7
:101E400005D1E368184214BF01200020E5E7002A0D
:101E5000EDD0F6E70028004010B5074BCA245C62BD
:101E60000A43B0F5807F4FF053045C620CBF5A64A4
:101E70009A64FF225A6210BD00280040044BB0F55E
:101E8000807F0CBF586C986CC0F30E00704700BF89
:101E900000280040074BCA225A6253225A629A68AD
:101EA00022F007029A609A681043FF2298605A62F3
:101EB000704700BF00280040044BCA225A625322D8
:101EC0005A62FF2258615A62704700BF00280040E2
:101ED000014B586980B270470028004082B000234F
:101EE0000193124BCA225A6253225A629A6840B135
:101EF00042F480629A6001200C4BFF225A6202B0C9
:101F0000704722F480629A601846DA6801990131BC
:101F100001910199B1F5005F02F0040201D0002A9D
:101F2000F3D0C068C0F38000E6E700BF002800409F
:101F3000074BCA225A6253225A629A6822F48022BC
:101F40009A609A6811430143FF2299605A62704770
:101F500000280040024B986800F48020704700BFC2
:101F600000280040074BCA225A6253225A629A68DC
:101F700022F4E0029A609A6811430143FF229960BB
:101F80005A62704700280040074BCA225A62532207
:101F90005A629A6828B142F400029A60FF225A629B
:101FA000704722F40002F8E700280040074BCA22DD
:101FB0005A6253225A629A6822F400229A609A68FE
:101FC0001043FF2298605A62704700BF002800400B
:101FD0000E4B30B5CA245C6253245C62DC68E403B7
:101FE00006D541F20104DD68ED0301D5013CFAD1CB
:101FF000064BDC68E4035CBF114308434FF0FF026B
:1020000056BFD863002001205A6230BD002800402E
:10201000084A936823F4006323F0080309B143F4EA
:102020000063CA2151620343532151629360FF232D
:102030005362704700280040204B2DE9F0411E6B91
:102040005D6B06F07F3727F0FE473C0C25F07F43A1
:1020500004F03F0E04F04004CC7023F0C0030024D1
:10206000C7F3062706F07F0681F800E04F708E70F8
:10207000C3F30428D47005F03F05C3F3423482F85B
:10208000018095701470B8B97046FFF748FC08706D
:102090003846FFF744FC48703046FFF740FC887034
:1020A0004046FFF73CFC50702846FFF738FC907024
:1020B0002046FFF734FC1070BDE8F0810028004096
:1020C000014B986B704700BF00280040044B400054
:1020D0001A6C19B922EA0000186470471043FBE734
:1020E00000280040044B1A6C11B11043186470476B
:1020F00022EA0000FAE700BF00280040044B1A6CF7
:1021000022F4C0521A641A6C10431864704700BF5E
:1021100000280040044B1A6C22F4E0621A641A6C26
:1021200010431864704700BF00280040044B1A6C2D
:1021300022F4C0421A641A6C10431864704700BF3E
:1021400000280040044B1A6C18B142F080021A6457
:10215000704722F08002FAE700280040044B1A6C16
:1021600018B122F400421A64704742F40042FAE7C0
:102170000028004082B000230193054B0193019B8E
:1021800003EB80000190019B196002B0704700BF13
:102190005028004082B000230193054B0193019B1E
:1021A00003EB80000190019B186802B0704700BFEC
:1021B00050280040044B1A6C22F480221A641A6CD6
:1021C00010431864704700BF00280040134BCA2218
:1021D00010B55A6253225A62DA68120706D542F2E3
:1021E0000102DC68240701D5013AFAD10B4AD36811
:1021F00013F008030DD19468E4060CD40143D162B6
:10220000FFF7F2FB003018BF0120044BFF225A6297
:1022100010BD0020F9E71846F7E700BF002800408E
:102220000D4BCA225A6253225A6220F0040200F077
:10223000040049B199680A439A601A6C1043186403
:10224000054BFF225A627047996821EA02029A60A0
:102250001A6C22EA0000F2E700280040044BDA681A
:10226000044B1340034214BF01200020704700BFFD
:10227000002800407FFF01000549064ACB68024064
:1022800042F0800203F0800363EA0203CB607047F0
:10229000002800407FFF01000B490B6C8A68C96869
:1022A00010B5840C20FA04F403F0040303EAD433D9
:1022B0000240134306D08BB213EA101314BF01205F
:1022C000002010BD184610BD00280040054AD36804
:1022D000C0F30F1040F0800003F0800363EA0003B6
:1022E000D36070470028004008B5154B98420BD1C9
:1022F00001214FF48050FFF79BFA00214FF48050EA
:10230000BDE80840FFF794BA0E4B98420BD101216B
:102310004FF48040FFF798FA00214FF48040BDE869
:102320000840FFF791BA084B984208D101214FF4B9
:102330000040FFF789FA00214FF40040EFE708BDA5
:102340000030014000380040003C00400023038082
:1023500043804FF4E062C380038143818381C38162
:1023600007238280038270472DE9F0474C88B1F83B
:1023700000A0B1F80680B1F808C0B1F80AE08F8972
:10238000CE898D88B4F5827F22D1028802F4415231
:1023900042EA0A0242F4827242EA080343EA0C0368
:1023A00043EA0E033B4333439BB20380838823F409
:1023B00070631B041B0C1D43ADB28580838B23F41B
:1023C00000631B041B0C83830B8A0382BDE8F08728
:1023D000B0F8049029F470694FEA09494FEA1949A5
:1023E00049EA0505ADB28580038803F441532343D0
:1023F00043EA0A0343EA080343EA0C0343EA0E03F1
:102400003B4333439BB20380D8E70023022203807F
:1024100043808380C380826083817047838B23F4F1
:102420007B6323F00F031B04F0B51B0C8383022393
:1024300003848B68868B022B91B005460C46B6B29E
:1024400039D08B8801A8002B14BF02270127FFF782
:1024500023F8E3880199A068B3F5007F4FF00A02E2
:1024600016BF7B010B0AB1FBF3F35343B3FBF0F34D
:1024700005330A229BB2B3FBF2F303F0010212020E
:10248000C3F34F03991E89B2FE2924BF0022022301
:102490001343E28813439BB262882B84238813433F
:1024A000A28843F400631343A28913431E43B6B2C8
:1024B000AE8311B0F0BD0022E4E7038821B19BB2E6
:1024C00043F040030380704723F040031B041B0CC0
:1024D000F8E7838821B19BB243F0100383807047F3
:1024E00023F010031B041B0CF8E7838B21B19BB274
:1024F00043F480638383704723F480631B041B0CC5
:10250000F8E7838823F470631B041B0C1943818054
:102510007047838823F480531B041B0C83808388BB
:102520009BB21943818070470388B1F5804F15BF76
:1025300023F480439BB21B0443F4804318BF1B0C5D
:10254000038070474FF6FF63994203880BBF23F463
:1025500080739BB21B0443F4807308BF1B0C038081
:102560007047838B0A8823F47B6323F00F031B04DB
:102570001B0C83830223038430B54B888D888989A3
:10258000848B2B4322F4007243F4006392B20B431A
:10259000002A43EA04030CBF4FF4807200229BB26E
:1025A0001343838330BD838821B19BB243F004037E
:1025B0008380704723F004031B041B0CF8E7838817
:1025C00021B19BB243F008038380704723F00803D6
:1025D0001B041B0CF8E70173704781817047007B77
:1025E0007047808980B27047038823F400631B041E
:1025F0001B0C038003889BB219430180704703883A
:1026000021B19BB243F400530380704723F400537D
:102610001B041B0CF8E703889BB243F48053038030
:102620007047012914BF008B808A80B27047008AEE
:1026300080B2704783889BB212B119438180704782
:1026400023EA0101FAE7838823F4C0431B041B0C2F
:10265000838083889BB21943818070470B090121D5
:102660009940838889B29BB212B119438180704727
:1026700023EA0101FAE7008900F4C050704700899D
:1026800000F4C06070470389194214BF0120002084
:102690007047C94389B20181704710B584880089A9
:1026A00001F00F02012380B203FA02F21040A4B23B
:1026B00005D009098B401C4214BF0120002010BD29
:1026C000084B1A6802F003021A601A6842F0F842D6
:1026D0001A6000225A609A60DA601A615A619A613F
:1026E000704700BF00000140034A136823F0030352
:1026F00018431060704700BF00000140044B1A6887
:1027000022F440021A601A6810431860704700BF34
:1027100000000140014B1860704700BF14002042C8
:10272000044B1A6811B110431860704722EA000088
:10273000FAE700BF00000140FFF7F2BFFFF7F0BF6C
:10274000FFF7EEBF01F0030301F0FC0101F180414E
:1027500001F5803110B58A689B000F249C4022EA65
:1027600004028A608A6898401043886010BD024B5A
:1027700001221A60704700BF10032042024A5368CA
:1027800018435060704700BF00000140024B986939
:10279000C0F30020704700BF00000140024A936967
:1027A00018439061704700BF00000140FFF7F6BF7B
:1027B00030B5046A24F0010404628569046A25F0D6
:1027C000F30542EA031324F00A0441F001012B430C
:1027D00021438361016230BD30B5046A24F01004E6
:1027E0002404240C04628569046A090124F0A0040D
:1027F0001202240441F0100125F4734542EA033328
:10280000240C89B22B4321438361016230BD08B59A
:102810003A4B98420BD101214FF40060FFF708F8C2
:1028200000214FF40060BDE80840FFF701B8B0F1A7
:10283000804F09D101210846FFF706F80021012049
:10284000BDE80840FFF700B82D4B984206D10121A2
:102850000220FEF7F9FF00210220F1E7294B984200
:1028600006D101210420FEF7EFFF00210420E7E755
:10287000254B984206D101211020FEF7E5FF0021EB
:102880001020DDE7214B984206D101212020FEF7E0
:10289000DBFF00212020D3E71D4B984208D1012106
:1028A0004FF40050FEF7C4FF00214FF40050BAE788
:1028B000184B984208D101214FF48030FEF7B8FF41
:1028C00000214FF48030AEE7134B984208D101212C
:1028D0004FF40030FEF7ACFF00214FF40030A2E7C8
:1028E0000E4B984208D101214FF48020FEF7A0FF43
:1028F00000214FF4802096E708BD00BF002C014066
:102900000004004000080040001000400014004097
:1029100000340140004001400044014000480140B3
:10292000204A038890429BB20ED002F5006290428A
:102930000AD0B0F1804F07D0A2F59832904203D070
:1029400002F58062904203D14A8823F0700313435A
:10295000154A904208D002F5806290421FBF23F4CE
:1029600040730A899BB2134303804B68C3620B8890
:1029700003850C4B98420FD003F5006398420BD0AF
:1029800003F54063984207D003F58063984203D073
:1029900003F58063984201D18B7A0386012343615A
:1029A000704700BF002C0140001000404FF0FF3383
:1029B0004360002303800381438083727047018555
:1029C00042617047038823F070031B041B0C1943FA
:1029D0000180704741627047C1627047406A70472A
:1029E000008D80B27047038821B19BB243F002038F
:1029F0000380704723F002031B041B0CF8E70388D5
:102A000021B19BB243F004030380704723F0040319
:102A10001B041B0CF8E7038821B19BB243F400634D
:102A20000380704723F400631B041B0CF8E7038842
:102A300021B19BB243F080030380704723F08003F1
:102A40001B041B0CF8E7038823F008031B041B0C72
:102A5000038003889BB2194301807047038823F4E5
:102A600040731B041B0C038003889BB21943018035
:102A70007047038821B19BB243F001030380704784
:102A800023F001031B041B0CF8E7036A23F0010386
:102A9000036270B5056A426884690B688E8824F405
:102AA000803424F073041C438B89334325F00205E2
:102AB0009BB22B43134DA8420FD005F50065A842E9
:102AC0000BD005F54065A84207D005F58065A84202
:102AD00003D005F58065A8420ED123F00805CB8907
:102AE0004E8A2B43CD8823F004032B4322F44075F8
:102AF0000A8A324392B22A4342608A6884614263FE
:102B0000036270BD002C0140036A23F010030362CE
:102B1000036A426830B584690D6824F0807424F437
:102B2000E64444EA05248D8923F0200343EA051393
:102B30008D8843EA05130F4DA84203D005F50065C3
:102B4000A84211D1CD8923F0800343EA0513CD8833
:102B500023F0400343EA05130D8A22F4406242EA5F
:102B600085024D8A42EA850242608A6884618263F6
:102B7000036230BD002C0140036A23F480730362BA
:102B8000036A426830B5C4690D6824F073042C43AD
:102B90008D8923F4007343EA05238D8843EA0523D6
:102BA0000F4DA84203D005F50065A84211D1CD898B
:102BB00023F4006343EA0523CD8823F4806343EACA
:102BC00005230D8A22F4405242EA05124D8A42EA58
:102BD000051242608A68C461C263036230BD00BFEF
:102BE000002C0140036A23F480530362036A30B56A
:102BF0004468C2690D6822F4E64242EA05228D89E2
:102C000023F4005343EA05338D8843EA0533094D25
:102C1000A84203D005F50065A84204D10D8A24F42A
:102C2000804444EA85144460C2618A680264036295
:102C300030BD00BF002C0140036A23F480330362DF
:102C4000036A30B54468426D0D6822F070022A4371
:102C50008D8923F4003343EA05438D8843EA054315
:102C6000084DA84203D005F50065A84204D10D8A9D
:102C700024F4803444EA0544446042658A688265ED
:102C8000036230BD002C0140036A23F48013036209
:102C9000036A30B54468426D0D6822F4E04242EAAE
:102CA00005228D8923F4001343EA05538D8843EAF6
:102CB0000553074DA84203D005F50065A84201D190
:102CC00024F40034446042658A68C265036230BD02
:102CD000002C0140836D19B143F0005383657047A8
:102CE00023F00053FAE7836D19B143F08043836505
:102CF000704723F08043FAE7836D19B143F0004336
:102D00008365704723F00043FAE700230360838064
:102D1000C38083608381C381038243827047012320
:102D20008B4030B5DB43056A9BB22B40036221F038
:102D3000080300F1180453B949080B5923F48033F0
:102D400023F070030B510B591A430A5130BD04395B
:102D5000490812020B5923F0807323F4E0430B510E
:102D600092B20B59F0E74163704781637047C163CA
:102D700070470164704781657047C165704783691A
:102D800023F4803323F07003194381617047836912
:102D900023F0807323F4E04343EA0121816170470B
:102DA000C36923F070031943C1617047C36923F4F9
:102DB000E04343EA0121C1617047436D23F0700392
:102DC000194341657047436D23F4E04343EA012111
:102DD00041657047836923F0080319438161704797
:102DE000836923F4006343EA012181617047C36969
:102DF00023F008031943C1617047C36923F40063DA
:102E000043EA0121C1617047436D23F00803194370
:102E100041657047436D23F4006343EA0121416536
:102E20007047836923F00403194381617047836904
:102E300023F4806343EA012181617047C36923F071
:102E400004031943C1617047C36923F4806343EAF3
:102E50000121C1617047836923F0800319438161B7
:102E60007047836923F4004343EA0121816170477D
:102E7000C36923F080031943C1617047C36923F418
:102E8000004343EA0121C1617047436D23F0800391
:102E9000194341657047436D23F4004343EA012120
:102EA00041657047836823F008031B041B0C836093
:102EB0008368194381607047036A23F00203194352
:102EC00001627047036A23F00803194301627047E7
:102ED000036A23F0200343EA011101627047036A89
:102EE00023F0800343EA011101627047036A23F46F
:102EF000007343EA012101627047036A23F400630F
:102F000043EA012101627047036A23F4005343EA54
:102F1000013101627047036A23F4003343EA01413F
:102F200001627047036A23F4001343EA015101620E
:102F30007047036A10B501248C4023EA040303623E
:102F4000036A8A401A43026210BD036A10B5042462
:102F50008C4023EA04030362036A8A401A43026234
:102F600010BD00230122038043808280C38003813F
:102F70007047406B7047806B7047C06B7047006C48
:102F80007047836923F00C0383618369194381616E
:102F90007047836923F440638361836943EA0121B5
:102FA00081617047F8B50C464988A288B4F800E002
:102FB000238900290CBF02260026012A0CBF022704
:102FC0000127BEF1000F0ED1FFF7F2FBE188FFF7FA
:102FD000D8FF314623893A46FFF7FEFBE188BDE87A
:102FE000F840FFF7D6BFFFF7F7FBE188FFF7D1FF07
:102FF000314623893A46FFF7DBFBE188BDE8F8401C
:10300000FFF7BFBFC36923F00C031B041B0CC36194
:10301000C3691943C1617047C36923F440631B044A
:103020001B0CC361C369090289B21943C1617047AE
:10303000F8B50E880B898A880D46498836B9FFF79E
:10304000B7FBE988BDE8F840FFF79BBF042E06D127
:10305000FFF7C2FBE988BDE8F840FFF79ABF082EEA
:10306000EF88056A1CD125F480752D042D0C0562AE
:10307000C669056AB6B2ADB226F0F30646EA031693
:1030800025F4206343EA0123B6B29BB2324343F4F2
:103090008073C26139460362BDE8F840FFF7B2BFF2
:1030A00025F480552D042D0C0562C669056A26F4A9
:1030B000407625F4005536056D04360D6D0C46EA54
:1030C000022245EA013189B242EA03339BB241F45C
:1030D0008051C36101623946BDE8F840FFF79CBFEB
:1030E0004A880B8813438A881343CA8813430A8982
:1030F00013434A8913438A8913439BB2436470473D
:10310000436C23F472234364436C43EA02420A4350
:1031100042647047436C23F03C734364436C43EA5E
:1031200002520A4342647047436C19B143F480531E
:103130004364704723F48053FAE7436C19B143F0BA
:1031400080734364704723F08073FAE700230380A1
:1031500043808380C3800381438183817047436CB4
:1031600019B143F4004343647047C3F30E03FAE715
:10317000436819B143F004034360704723F004032C
:103180001B041B0CF8E7436819B143F001034360CB
:10319000704723F001031B041B0CF8E741617047E3
:1031A00003690B4214BF012000207047C94389B254
:1031B000016170470369C26811EA030003D011423C
:1031C00014BF012000207047C94389B201617047D4
:1031D0000A43A0F848207047C36812B11943C16080
:1031E0007047C94389B21940F9E7FFF7F5BF436853
:1031F00019B143F008034360704723F008031B0430
:103200001B0CF8E7836823F007031B041B0C836087
:10321000704782684FF68F7313401943816083684B
:1032200043F007038360704738B50D46602D1146A3
:1032300004464FF001020CD1FFF7CEFAA2684FF618
:103240008F7313401D43A560A36843F00703A36079
:1032500038BDFFF7ADFAF1E782684FF68F73134080
:10326000194381607047436823F070031B041B0CF3
:1032700043604368194341607047436823F4700317
:1032800043604368194341607047836823F4803387
:1032900023F0070383608368194381607047836864
:1032A00023F080031B041B0C836083681943816037
:1032B000704710B584680A43E4B242EA03231C4312
:1032C000A4B2846010BD10B5FFF7F3FF836823F04C
:1032D00077039BB243F07703836010BD10B5FFF70F
:1032E000E8FF836843F48043836010BDF0B58568D0
:1032F0008469076A4FF6F8762E404FF6FC45254064
:103300004FF6DD743C4042EA031345F480751C43DC
:10331000314345F00105A4B2816085610462F0BDCE
:10332000436819B143F080034360704723F0800382
:103330001B041B0CF8E7A0F85010704708B5214B90
:1033400098420BD101214FF48040FEF771FA002121
:103350004FF48040BDE80840FEF76ABA1A4B984225
:103360000BD101214FF40030FEF76EFA00214FF42B
:103370000030BDE80840FEF767BA144B984208D108
:1033800001214FF48020FEF75FFA00214FF48020E6
:10339000EFE70F4B984208D101214FF40020FEF7D0
:1033A00053FA00214FF40020E3E70A4B984208D17A
:1033B00001214FF48010FEF747FA00214FF48010EE
:1033C000D7E708BD003801400044004000480040F5
:1033D000004C00400050004003688A6823F001035D
:1033E00030B50360436823F44053134343600D46F4
:1033F0004B68C96802680B43296922F4B05222F075
:103400000C020B431343036083686A6923F440731F
:10341000134391B08360044601A8FEF73DF8184BB2
:103420009C421CD10B9A2368296813F4004F18BFE3
:103430005200B2FBF1F301FB1322B2EB510F2268F1
:1034400028BF0133120406D5C3F3420223F00F0351
:103450001B041B0C13439BB2A38111B030BD094B5D
:103460009C4201D10C9ADEE7074B9C4201D10D9A98
:10347000D9E7064B9C420CBF0E9A0F9AD3E700BFC8
:10348000003801400044004000480040004C00402B
:103490004FF4165303600C22002343608360C36023
:1034A00002614361704710B591E8180023438C68AE
:1034B0004268C968234322F470620B43134343609C
:1034C00010BD0023036043608360C36070470368DE
:1034D00019B143F001030360704723F00103FAE7D9
:1034E000036812B119430160704723EA0101FAE74A
:1034F000036819B143F400430360704723F40043A9
:10350000FAE7836819B143F400638360704723F4DA
:103510000063FAE7436819B143F40023436070473E
:1035200023F40023FAE7436819B143F4802343608E
:10353000704723F48023FAE7436812B119434160CE
:10354000704723EA0101FAE7436819B143F40043E5
:103550004360704723F40043FAE7436819B143F42A
:1035600000034360704723F40003FAE7436903F064
:103570007F4343614369194341617047038A03F400
:103580007F430382038A9BB2194301827047036819
:1035900019B143F002030360704723F00203FAE716
:1035A000836823F440138360836819438160704704
:1035B000436819B143F480134360704723F48013C8
:1035C000FAE7436823F4C00343604368194341604A
:1035D0007047C1F3080101857047808CC0F3080073
:1035E0007047436823F07F434360436843EA0161C7
:1035F00041607047036819B143F40053036070479A
:1036000023F40053FAE7036823F4006303600368BC
:10361000194301607047436823F010034360436817
:10362000194341607047436823F0200343604368B7
:10363000194341607047436819B143F480434360C4
:10364000704723F48043FAE7836819B143F0080315
:103650008360704723F00803FAE7038ADBB2038232
:10366000038A9BB243EA012101827047836819B142
:1036700043F020038360704723F02003FAE7836858
:1036800019B143F010038360704723F01003FAE789
:10369000836823F460238360836843EA4141816047
:1036A0007047436923F07F434361436943EA016103
:1036B00041617047836823F0040383608368194382
:1036C00081607047836819B143F0020383607047DB
:1036D00023F00203FAE7836819B143F4804383605F
:1036E000704723F48043FAE7836823F40043836040
:1036F0008368194381607047036823F0787303601F
:10370000036843EA415101607047036823F4F813EA
:103710000360036843EA014101607047836812B1A6
:1037200019438160704723EA0101FAE7836823F4B3
:1037300000538360836819438160704710B5C1F3FB
:103740000724CBB2022C4FF0010101FA03F105D19D
:103750000430036832B11943016010BD032C08BF67
:103760000830F6E723EA0101F6E7038B1AB11943A3
:1037700089B2018370479BB223EA0101F9E78368AC
:1037800023F4805383608368194381607047C36961
:103790000B4214BF01200020704701627047C1F343
:1037A000072210B50123CCB2012A03FA04F30CD18D
:1037B00002681340C2696BB10123090C03FA01F1DD
:1037C000114214BF1846002010BD022A0CBF4268E7
:1037D0008268EEE7184610BD090C012303FA01F1D7
:1037E0000162704781F0004102E000BF83F00043B6
:1037F00030B54FEA41044FEA430594EA050F08BF8C
:1038000090EA020F1FBF54EA000C55EA020C7FEA4F
:10381000645C7FEA655C00F0E2804FEA5454D4EBCC
:103820005555B8BF6D420CDD2C4480EA020281EA96
:10383000030382EA000083EA010180EA020281EACE
:103840000303362D88BF30BD11F0004F4FEA013120
:103850004FF4801C4CEA113102D0404261EB41012F
:1038600013F0004F4FEA03334CEA133302D05242B5
:1038700063EB430394EA050F00F0A780A4F1010471
:10388000D5F1200E0DDB02FA0EFC22FA05F28018AB
:1038900041F1000103FA0EF2801843FA05F3594191
:1038A0000EE0A5F120050EF1200E012A03FA0EFC10
:1038B00028BF4CF0020C43FA05F3C01851EBE3713A
:1038C00001F0004507D54FF0000EDCF1000C7EEB57
:1038D00000006EEB0101B1F5801F1BD3B1F5001F95
:1038E0000CD349085FEA30004FEA3C0C04F10104B4
:1038F0004FEA445212F5800F80F09A80BCF1004FDD
:1039000008BF5FEA500C50F1000041EB045141EA5E
:10391000050130BD5FEA4C0C404141EB010111F45F
:10392000801FA4F10104E9D191F0000F04BF01460A
:103930000020B1FA81F308BF2033A3F10B03B3F1E8
:1039400020020CDA0C3208DD02F1140CC2F10C0278
:1039500001FA0CF021FA02F10CE002F11402D8BFD6
:10396000C2F1200C01FA02F120FA0CFCDCBF41EAA2
:103970000C019040E41AA2BF01EB0451294330BD71
:103980006FEA04041F3C1CDA0C340EDC04F114044E
:10399000C4F1200220FA04F001FA02F340EA030025
:1039A00021FA04F345EA030130BDC4F10C04C4F16B
:1039B000200220FA02F001FA04F340EA030029464B
:1039C00030BD21FA04F0294630BD94F0000F83F495
:1039D000801306BF81F480110134013D4EE77FEA78
:1039E000645C18BF7FEA655C29D094EA050F08BFC4
:1039F00090EA020F05D054EA000C04BF19461046A5
:103A000030BD91EA030F1EBF0021002030BD5FEAE8
:103A1000545C05D14000494128BF41F0004130BD10
:103A200014F580043CBF01F5801130BD01F0004564
:103A300045F0FE4141F470014FF0000030BD7FEAD7
:103A4000645C1ABF194610467FEA655C1CBF0B46D2
:103A5000024650EA013406BF52EA033591EA030FE9
:103A600041F4002130BD00BF90F0000F04BF0021E1
:103A7000704730B54FF4806404F132044FF0000514
:103A80004FF0000150E700BF90F0000F04BF00218D
:103A9000704730B54FF4806404F1320410F00045F3
:103AA00048BF40424FF000013EE700BF42004FEAEE
:103AB000E2014FEA31014FEA02701FBF12F07F436B
:103AC00093F07F4F81F06051704792F0000F14BF68
:103AD00093F07F4F704730B54FF4607401F00045AC
:103AE00021F0004120E700BF50EA010208BF704703
:103AF00030B54FF000050AE050EA010208BF7047F8
:103B000030B511F0004502D5404261EB41014FF460
:103B1000806404F132045FEA915C3FF4DCAE4FF064
:103B200003025FEADC0C18BF03325FEADC0C18BF4B
:103B3000033202EBDC02C2F1200300FA03FC20FA9C
:103B400002F001FA03FE40EA0E0021FA02F11444E9
:103B5000C1E600BF70B54FF0FF0C4CF4E06C1CEAFE
:103B600011541DBF1CEA135594EA0C0F95EA0C0F73
:103B700000F0DEF82C4481EA030621EA4C5123EAE6
:103B80004C5350EA013518BF52EA033541F4801115
:103B900043F4801338D0A0FB02CE4FF00005E1FBC8
:103BA00002E506F00042E0FB03E54FF00006E1FB12
:103BB00003569CF0000F18BF4EF0010EA4F1FF0455
:103BC000B6F5007F64F5407404D25FEA4E0E6D4195
:103BD00046EB060642EAC62141EA55514FEAC520A6
:103BE00040EA5E504FEACE2EB4F1FD0C88BFBCF522
:103BF000E06F1ED8BEF1004F08BF5FEA500E50F1D3
:103C0000000041EB045170BD06F0004646EA010198
:103C100040EA020081EA0301B4EB5C04C2BFD4EBCA
:103C20000C0541EA045170BD41F480114FF0000EC3
:103C3000013C00F3AB8014F1360FDEBF002001F031
:103C4000004170BDC4F10004203C35DA0C341BDCAB
:103C500004F11404C4F1200500FA05F320FA04F07D
:103C600001FA05F240EA020001F0004221F00041B1
:103C700010EBD37021FA04F642EB06015EEA430E24
:103C800008BF20EAD37070BDC4F10C04C4F1200554
:103C900000FA04F320FA05F001FA04F240EA020007
:103CA00001F0004110EBD37041F100015EEA430ED8
:103CB00008BF20EAD37070BDC4F1200500FA05F2F8
:103CC0004EEA020E20FA04F301FA05F243EA020377
:103CD00021FA04F001F0004121FA04F220EA020086
:103CE00000EBD3705EEA430E08BF20EAD37070BDCC
:103CF00094F0000F0FD101F00046400041EB0101AC
:103D000011F4801F08BF013CF7D041EA060195F08D
:103D1000000F18BF704703F00046520043EB030347
:103D200013F4801F08BF013DF7D043EA0603704734
:103D300094EA0C0F0CEA135518BF95EA0C0F0CD03F
:103D400050EA410618BF52EA4306D1D181EA030185
:103D500001F000414FF0000070BD50EA410606BF7F
:103D60001046194652EA430619D094EA0C0F02D1C4
:103D700050EA013613D195EA0C0F05D152EA033609
:103D80001CBF104619460AD181EA030101F0004127
:103D900041F0FE4141F470014FF0000070BD41F070
:103DA000FE4141F4780170BD70B54FF0FF0C4CF44A
:103DB000E06C1CEA11541DBF1CEA135594EA0C0F69
:103DC00095EA0C0F00F0A7F8A4EB050481EA030EB6
:103DD00052EA03354FEA013100F088804FEA03339D
:103DE0004FF0805545EA131343EA12634FEA02226B
:103DF00045EA111545EA10654FEA00260EF000412C
:103E00009D4208BF964244F1FD0404F5407402D27D
:103E10005B084FEA3202B61A65EB03055B084FEA0E
:103E200032024FF480104FF4002CB6EB020E75EB0B
:103E3000030E22BFB61A754640EA0C005B084FEA33
:103E40003202B6EB020E75EB030E22BFB61A7546B0
:103E500040EA5C005B084FEA3202B6EB020E75EBFB
:103E6000030E22BFB61A754640EA9C005B084FEA73
:103E70003202B6EB020E75EB030E22BFB61A754680
:103E800040EADC0055EA060E18D04FEA051545EA6F
:103E900016754FEA06164FEAC30343EA52734FEA18
:103EA000C2025FEA1C1CC0D111F4801F0BD141EA91
:103EB00000014FF000004FF0004CB6E711F4801FF6
:103EC00004BF01430020B4F1FD0C88BFBCF5E06FD6
:103ED0003FF6AFAEB5EB030C04BFB6EB020C5FEAE6
:103EE000500C50F1000041EB045170BD0EF0004E3B
:103EF0004EEA113114EB5C04C2BFD4EB0C0541EA6D
:103F0000045170BD41F480114FF0000E013C90E669
:103F100045EA060E8DE60CEA135594EA0C0F08BF2D
:103F200095EA0C0F3FF43BAF94EA0C0F0AD150EA2C
:103F300001347FF434AF95EA0C0F7FF425AF1046BF
:103F400019462CE795EA0C0F06D152EA03353FF4E7
:103F5000FDAE1046194622E750EA410618BF52EA64
:103F600043067FF4C5AE50EA41047FF40DAF52EA38
:103F700043057FF4EBAE12E74FEA410212F500125F
:103F800015D211D56FF47873B3EB625212D94FEAA0
:103F9000C12343F0004343EA505311F0004F23FA8A
:103FA00002F018BF404270474FF00000704750EADF
:103FB000013005D111F0004008BF6FF0004070479C
:103FC0004FF00000704700BF4FEA4102B2F1E043FA
:103FD00024BFB3F5001CDCF1FE5C0DD901F0004CF0
:103FE0004FEAC0024CEA5070B2F1004F40EB830040
:103FF00008BF20F00100704711F0804F21D113F16C
:104000003872BCBF01F00040704741F480114FEAA4
:104010005252C2F11802C2F1200C10FA0CF320FA2D
:1040200002F018BF40F001004FEAC1234FEAD3234A
:1040300003FA0CFC40EA0C0023FA02F34FEA4303B4
:10404000CCE77FEA625307D150EA01331EBF4FF03D
:10405000FE4040F44000704701F0004040F0FE4058
:1040600040F40000704700BF002103E00A4B5B589A
:104070004350043109480A4B42189A42F6D3094A80
:1040800002E0002342F8043B074B9A42F9D3FBF7C6
:10409000D1FD00F00DF87047BC420108000000207F
:1040A000A4000020A400002014340020FEE700003B
:1040B0002F49CA6822F4E06208B512042D4B120C95
:1040C0001343CB604FF080500121FDF799FB012194
:1040D0000846FDF789FB62B6274CF4F738F9F4F788
:1040E00095FDF4F7D1F8FBF7EFFBFBF7DDFCF4F7F8
:1040F000DCFFF4F747FA2078F4F7FCFBE078F4F7FC
:104100005FFDF5F7EFFDF5F7DBF9FAF7ADFF1B4BB8
:10411000DC699CB10120FBF739F9F6F7A9FDF9F745
:1041200003FB174B4FF000629A61F9F77DF8F9F73E
:10413000FCFAF9F709FCFBF7BFF9F6E7114D224647
:1041400020466021F5F70BFD224620466121F5F758
:1041500006FDEA891C212046F5F701FD6868FBF79A
:10416000D9F8A868FBF7E8F8287BFBF7FDF8D4E757
:1041700000ED00E00007FA0504000020902E00206A
:1041800000040048D02E002010B5431E0A4491427E
:1041900000D110BD11F8014B03F8014FF7E7614062
:1041A00001AA80000020C08000002B2001AA80000E
:1041B0000020C0800000000000000000E093040028
:1041C000C0270900FF00FE000000000032FF0000D1
:1041D000E80300001027000088130000D00700004B
:1041E0000A0000000000000000C2EB0B000001000C
:1041F000640000006400000000070000F4010000FB
:104200000000000000000000E0930400C027090047
:10421000FF00FE000000000064F00000E803000062
:104220001027000010270000140000000A00000002
:1042300000000000FFFFFF3F0000010064000000DD
:104240006400000000070000F4010000000000000E
:104250000050C3000088130001400808000000005F
:1042600000000000C8000000010000000000000085
:10427000000000000000000000000000000000003E
:10428000000000000000000000000000000100002D
:10429000313337305631333500000000F8B500BFF8
:1042A000F8BC08BC9E467047F8B500BFF8BC08BC17
:0442B0009E4670476F
:0442B400AD810008D0
:0442B80089810008F0
:1042BC00904201080001020000080000010000000B
:1042CC0002000000000000000000000000000000E0
:1042DC0000000000000000000000000000000000D2
:1042EC0000000000000000000000000000000000C2
:1042FC000000000002000000C0270900E093040049
:10430C0001000000010000000A0000002003000072
:10431C005100000000A24A04000000000000000050
:10432C00010203040607080900000000010203044F
:10433C000102030406070809000001000200040042
:10434C00060008000A000C0010002000400080004D
:04435C00000100005C
:040000050801406945
:00000001FF
